 iterinstcls002

 Timestamp is 028e9fbe (reproducible build file hash)

 Preferred load address is 0000000180000000

 Start         Length     Name                   Class
 0001:00000000 00004c10H .text$mn                CODE
 0001:00004c10 00000036H .text$mn$00             CODE
 0001:00004c46 00000092H .text$x                 CODE
 0002:00000000 000001c8H .idata$5                DATA
 0002:000001c8 00000038H .00cfg                  DATA
 0002:00000200 00000008H .CRT$XCA                DATA
 0002:00000208 00000008H .CRT$XCZ                DATA
 0002:00000210 00000008H .CRT$XIA                DATA
 0002:00000218 00000008H .CRT$XIC                DATA
 0002:00000220 00000008H .CRT$XIZ                DATA
 0002:00000228 00000008H .CRT$XLA                DATA
 0002:00000230 00000008H .CRT$XLZ                DATA
 0002:00000238 00000008H .CRT$XPA                DATA
 0002:00000240 00000008H .CRT$XPZ                DATA
 0002:00000248 00000008H .CRT$XTA                DATA
 0002:00000250 00000010H .CRT$XTZ                DATA
 0002:00000258 00000000H .gehcont$y              DATA
 0002:00000258 00000000H .gfids$y                DATA
 0002:00000260 000031a0H .rdata                  DATA
 0002:00003400 00000000H .rdata$CastGuardVftablesA DATA
 0002:00003400 00000000H .rdata$CastGuardVftablesC DATA
 0002:00003400 00000028H .rdata$T                DATA
 0002:00003428 000000d0H .rdata$voltmd           DATA
 0002:000034f8 00000320H .rdata$zzzdbg           DATA
 0002:00003818 00000008H .rtc$IAA                DATA
 0002:00003820 00000008H .rtc$IZZ                DATA
 0002:00003828 00000008H .rtc$TAA                DATA
 0002:00003830 00000008H .rtc$TZZ                DATA
 0002:00003838 00000004H .tls                    DATA
 0002:0000383c 00000004H .tls$                   DATA
 0002:00003840 00000008H .tls$ZZZ                DATA
 0002:00003848 000003e8H .xdata                  DATA
 0002:00003c30 00000384H .edata                  DATA
 0002:00003fb4 0000008cH .idata$2                DATA
 0002:00004040 00000018H .idata$3                DATA
 0002:00004058 000001c8H .idata$4                DATA
 0002:00004220 00000486H .idata$6                DATA
 0003:00000000 00000080H .data                   DATA
 0003:00000080 0001b258H .bss                    DATA
 0004:00000000 0000042cH .pdata                  DATA

  Address         Publics by Value              Rva+Base               Lib:Object

 0000:00000000       __AbsoluteZero             0000000000000000     <absolute>
 0000:00000000       ___safe_se_handler_count   0000000000000000     <absolute>
 0000:00000000       ___safe_se_handler_table   0000000000000000     <absolute>
 0000:00000000       __arm64x_extra_rfe_table   0000000000000000     <absolute>
 0000:00000000       __arm64x_extra_rfe_table_size 0000000000000000     <absolute>
 0000:00000000       __arm64x_native_entrypoint 0000000000000000     <absolute>
 0000:00000000       __arm64x_redirection_metadata 0000000000000000     <absolute>
 0000:00000000       __arm64x_redirection_metadata_count 0000000000000000     <absolute>
 0000:00000000       __dynamic_value_reloc_table 0000000000000000     <absolute>
 0000:00000000       __enclave_config           0000000000000000     <absolute>
 0000:00000000       __guard_check_icall_a64n_fptr 0000000000000000     <absolute>
 0000:00000000       __guard_eh_cont_count      0000000000000000     <absolute>
 0000:00000000       __guard_eh_cont_table      0000000000000000     <absolute>
 0000:00000000       __guard_fids_count         0000000000000000     <absolute>
 0000:00000000       __guard_fids_table         0000000000000000     <absolute>
 0000:00000000       __guard_iat_count          0000000000000000     <absolute>
 0000:00000000       __guard_iat_table          0000000000000000     <absolute>
 0000:00000000       __guard_longjmp_count      0000000000000000     <absolute>
 0000:00000000       __guard_longjmp_table      0000000000000000     <absolute>
 0000:00000000       __hybrid_auxiliary_iat     0000000000000000     <absolute>
 0000:00000000       __hybrid_auxiliary_iat_copy 0000000000000000     <absolute>
 0000:00000000       __hybrid_code_map          0000000000000000     <absolute>
 0000:00000000       __hybrid_code_map_count    0000000000000000     <absolute>
 0000:00000000       __x64_code_ranges_to_entry_points 0000000000000000     <absolute>
 0000:00000000       __x64_code_ranges_to_entry_points_count 0000000000000000     <absolute>
 0000:00000100       __guard_flags              0000000000000100     <absolute>
 0000:00000000       __ImageBase                0000000180000000     <linker-defined>
 0001:00000000       ?NewObject@JNIEnv_@@QEAAPEAV_jobject@@PEAV_jclass@@PEAU_jmethodID@@ZZ 0000000180001000 f i libiterinstcls002.obj
 0001:00000028       ?SetEventNotificationMode@_jvmtiEnv@@QEAA?AW4jvmtiError@@W4jvmtiEventMode@@W4jvmtiEvent@@PEAV_jobject@@ZZ 0000000180001028 f i libiterinstcls002.obj
 0001:00000034       ?TranslateError@@YAPEBDW4jvmtiError@@@Z 0000000180001034 f   libiterinstcls002.obj
 0001:000002ec       ?nsk_jni_check_exception@@YAHPEAUJNIEnv_@@QEBDH@Z 00000001800012ec f   libiterinstcls002.obj
 0001:00000430       ?nsk_jni_lverify@@YAHHPEAUJNIEnv_@@HQEBDH1ZZ 0000000180001430 f   libiterinstcls002.obj
 0001:000004d0       Agent_Initialize           00000001800014d0 f   libiterinstcls002.obj
 0001:000008a4       Agent_OnAttach             00000001800018a4 f   libiterinstcls002.obj
 0001:000008a4       Agent_OnLoad               00000001800018a4 f   libiterinstcls002.obj
 0001:000008ac       Java_nsk_jvmti_unit_FollowReferences_FollowRefObjects_addRefToVerify 00000001800018ac f   libiterinstcls002.obj
 0001:00000a84       Java_nsk_jvmti_unit_FollowReferences_FollowRefObjects_getTag 0000000180001a84 f   libiterinstcls002.obj
 0001:00000b44       Java_nsk_jvmti_unit_FollowReferences_FollowRefObjects_resetRefsToVerify 0000000180001b44 f   libiterinstcls002.obj
 0001:00000b4c       Java_nsk_jvmti_unit_FollowReferences_FollowRefObjects_resetTags 0000000180001b4c f   libiterinstcls002.obj
 0001:00000b90       Java_nsk_jvmti_unit_FollowReferences_FollowRefObjects_setTag 0000000180001b90 f   libiterinstcls002.obj
 0001:00000de8       Java_nsk_share_jvmti_ArgumentHandler_getAgentOptionsString 0000000180001de8 f   libiterinstcls002.obj
 0001:00000e98       Java_nsk_share_jvmti_DebugeeClass_checkStatus 0000000180001e98 f   libiterinstcls002.obj
 0001:00000f20       Java_nsk_share_jvmti_DebugeeClass_resetAgentData 0000000180001f20 f   libiterinstcls002.obj
 0001:00000f80       Java_nsk_share_jvmti_RedefineAgent_agentStatus 0000000180001f80 f   libiterinstcls002.obj
 0001:00000f8c       Java_nsk_share_jvmti_RedefineAgent_isRedefined 0000000180001f8c f   libiterinstcls002.obj
 0001:00000f98       Java_nsk_share_jvmti_RedefineAgent_redefineAttempted 0000000180001f98 f   libiterinstcls002.obj
 0001:00000fa4       MA_checkStatus             0000000180001fa4 f   libiterinstcls002.obj
 0001:00001048       __local_stdio_printf_options 0000000180002048 f i libiterinstcls002.obj
 0001:0000166c       callbackObjectFree         000000018000266c f   libiterinstcls002.obj
 0001:00001abc       exitOnError                0000000180002abc f   libiterinstcls002.obj
 0001:00001b70       fprintf                    0000000180002b70 f i libiterinstcls002.obj
 0001:000027d0       heapObjectCallback         00000001800037d0 f   libiterinstcls002.obj
 0001:00002988       nsk_complain               0000000180003988 f   libiterinstcls002.obj
 0001:000029b4       nsk_jvmti_createJVMTIEnv   00000001800039b4 f   libiterinstcls002.obj
 0001:00002ae4       nsk_jvmti_enableEvents     0000000180003ae4 f   libiterinstcls002.obj
 0001:00002bb8       nsk_jvmti_findOptionIntValue 0000000180003bb8 f   libiterinstcls002.obj
 0001:00002c54       nsk_jvmti_findOptionValue  0000000180003c54 f   libiterinstcls002.obj
 0001:00002ccc       nsk_jvmti_lverify          0000000180003ccc f   libiterinstcls002.obj
 0001:00002dbc       nsk_jvmti_parseOptions     0000000180003dbc f   libiterinstcls002.obj
 0001:0000300c       nsk_jvmti_resetAgentData   000000018000400c f   libiterinstcls002.obj
 0001:0000308c       nsk_jvmti_resumeSync       000000018000408c f   libiterinstcls002.obj
 0001:00003134       nsk_jvmti_setFailStatus    0000000180004134 f   libiterinstcls002.obj
 0001:00003170       nsk_jvmti_waitForSync      0000000180004170 f   libiterinstcls002.obj
 0001:00003274       nsk_lcomplain              0000000180004274 f   libiterinstcls002.obj
 0001:00003294       nsk_ldisplay               0000000180004294 f   libiterinstcls002.obj
 0001:000032b4       nsk_ltrace                 00000001800042b4 f   libiterinstcls002.obj
 0001:000032d4       nsk_lvcomplain             00000001800042d4 f   libiterinstcls002.obj
 0001:0000348c       nsk_lvdisplay              000000018000448c f   libiterinstcls002.obj
 0001:000034d8       nsk_lverify                00000001800044d8 f   libiterinstcls002.obj
 0001:00003534       nsk_lvtrace                0000000180004534 f   libiterinstcls002.obj
 0001:00003594       nsk_printf                 0000000180004594 f   libiterinstcls002.obj
 0001:000035bc       nsk_vprintf                00000001800045bc f   libiterinstcls002.obj
 0001:00003670       printf                     0000000180004670 f i libiterinstcls002.obj
 0001:00003ce8       __raise_securityfailure    0000000180004ce8 f   MSVCRT:gs_report.obj
 0001:00003d1c       __report_gsfailure         0000000180004d1c f   MSVCRT:gs_report.obj
 0001:00003f5c       __GSHandlerCheck           0000000180004f5c f   MSVCRT:gshandler.obj
 0001:00003f7c       __GSHandlerCheckCommon     0000000180004f7c f   MSVCRT:gshandler.obj
 0001:00003ff0       __security_check_cookie    0000000180004ff0 f   MSVCRT:amdsecgs.obj
 0001:00004330       _DllMainCRTStartup         0000000180005330 f   MSVCRT:dll_dllmain.obj
 0001:00004370       __scrt_acquire_startup_lock 0000000180005370 f   MSVCRT:utility.obj
 0001:000043ac       __scrt_dllmain_after_initialize_c 00000001800053ac f   MSVCRT:utility.obj
 0001:000043e0       __scrt_dllmain_before_initialize_c 00000001800053e0 f   MSVCRT:utility.obj
 0001:000043f8       __scrt_dllmain_crt_thread_attach 00000001800053f8 f   MSVCRT:utility.obj
 0001:00004420       __scrt_dllmain_crt_thread_detach 0000000180005420 f   MSVCRT:utility.obj
 0001:00004438       __scrt_dllmain_exception_filter 0000000180005438 f   MSVCRT:utility.obj
 0001:00004498       __scrt_dllmain_uninitialize_c 0000000180005498 f   MSVCRT:utility.obj
 0001:000044c8       __scrt_dllmain_uninitialize_critical 00000001800054c8 f   MSVCRT:utility.obj
 0001:000044dc       __scrt_initialize_crt      00000001800054dc f   MSVCRT:utility.obj
 0001:00004528       __scrt_initialize_onexit_tables 0000000180005528 f   MSVCRT:utility.obj
 0001:000045b4       __scrt_is_nonwritable_in_current_image 00000001800055b4 f   MSVCRT:utility.obj
 0001:0000464c       __scrt_release_startup_lock 000000018000564c f   MSVCRT:utility.obj
 0001:00004670       __scrt_uninitialize_crt    0000000180005670 f   MSVCRT:utility.obj
 0001:0000469c       _onexit                    000000018000569c f   MSVCRT:utility.obj
 0001:000046d8       atexit                     00000001800056d8 f   MSVCRT:utility.obj
 0001:000046f0       __crt_debugger_hook        00000001800056f0 f   MSVCRT:utility_desktop.obj
 0001:000046f8       __scrt_fastfail            00000001800056f8 f   MSVCRT:utility_desktop.obj
 0001:00004844       _guard_check_icall_nop     0000000180005844 f i MSVCRT:guard_support.obj
 0001:00004848       __security_init_cookie     0000000180005848 f   MSVCRT:gs_support.obj
 0001:000048f4       DllMain                    00000001800058f4 f   MSVCRT:dll_dllmain_stub.obj
 0001:00004918       ?__scrt_initialize_type_info@@YAXXZ 0000000180005918 f   MSVCRT:tncleanup.obj
 0001:00004928       ?__scrt_uninitialize_type_info@@YAXXZ 0000000180005928 f   MSVCRT:tncleanup.obj
 0001:00004934       __local_stdio_scanf_options 0000000180005934 f i MSVCRT:default_local_stdio_options.obj
 0001:0000493c       __scrt_initialize_default_local_stdio_options 000000018000593c f   MSVCRT:default_local_stdio_options.obj
 0001:00004958       __scrt_get_dyn_tls_init_callback 0000000180005958 f   MSVCRT:dyn_tls_init.obj
 0001:00004960       _RTC_Initialize            0000000180005960 f   MSVCRT:initsect.obj
 0001:0000499c       _RTC_Terminate             000000018000599c f   MSVCRT:initsect.obj
 0001:000049d8       __isa_available_init       00000001800059d8 f   MSVCRT:cpu_disp.obj
 0001:00004b84       _get_startup_argv_mode     0000000180005b84 f   MSVCRT:argv_mode.obj
 0001:00004b8c       __scrt_is_ucrt_dll_in_use  0000000180005b8c f   MSVCRT:ucrt_detection.obj
 0001:00004ba0       memcpy                     0000000180005ba0 f   vcruntime:VCRUNTIME140.dll
 0001:00004ba6       memset                     0000000180005ba6 f   vcruntime:VCRUNTIME140.dll
 0001:00004bac       strchr                     0000000180005bac f   vcruntime:VCRUNTIME140.dll
 0001:00004bb2       __C_specific_handler       0000000180005bb2 f   vcruntime:VCRUNTIME140.dll
 0001:00004bb8       __std_type_info_destroy_list 0000000180005bb8 f   vcruntime:VCRUNTIME140.dll
 0001:00004bbe       strcmp                     0000000180005bbe f   ucrt:api-ms-win-crt-string-l1-1-0.dll
 0001:00004bc4       strlen                     0000000180005bc4 f   ucrt:api-ms-win-crt-string-l1-1-0.dll
 0001:00004bca       _initterm                  0000000180005bca f   ucrt:api-ms-win-crt-runtime-l1-1-0.dll
 0001:00004bd0       _initterm_e                0000000180005bd0 f   ucrt:api-ms-win-crt-runtime-l1-1-0.dll
 0001:00004bd6       _seh_filter_dll            0000000180005bd6 f   ucrt:api-ms-win-crt-runtime-l1-1-0.dll
 0001:00004bdc       _configure_narrow_argv     0000000180005bdc f   ucrt:api-ms-win-crt-runtime-l1-1-0.dll
 0001:00004be2       _initialize_narrow_environment 0000000180005be2 f   ucrt:api-ms-win-crt-runtime-l1-1-0.dll
 0001:00004be8       _initialize_onexit_table   0000000180005be8 f   ucrt:api-ms-win-crt-runtime-l1-1-0.dll
 0001:00004bee       _register_onexit_function  0000000180005bee f   ucrt:api-ms-win-crt-runtime-l1-1-0.dll
 0001:00004bf4       _execute_onexit_table      0000000180005bf4 f   ucrt:api-ms-win-crt-runtime-l1-1-0.dll
 0001:00004bfa       _crt_atexit                0000000180005bfa f   ucrt:api-ms-win-crt-runtime-l1-1-0.dll
 0001:00004c00       _cexit                     0000000180005c00 f   ucrt:api-ms-win-crt-runtime-l1-1-0.dll
 0001:00004c08       __acrt_initialize          0000000180005c08 f   MSVCRT:ucrt_stubs.obj
 0001:00004c08       __acrt_thread_attach       0000000180005c08 f   MSVCRT:ucrt_stubs.obj
 0001:00004c08       __acrt_thread_detach       0000000180005c08 f   MSVCRT:ucrt_stubs.obj
 0001:00004c08       __acrt_uninitialize        0000000180005c08 f   MSVCRT:ucrt_stubs.obj
 0001:00004c08       __acrt_uninitialize_critical 0000000180005c08 f   MSVCRT:ucrt_stubs.obj
 0001:00004c08       __scrt_stub_for_acrt_initialize 0000000180005c08 f   MSVCRT:ucrt_stubs.obj
 0001:00004c08       __scrt_stub_for_acrt_thread_attach 0000000180005c08 f   MSVCRT:ucrt_stubs.obj
 0001:00004c08       __scrt_stub_for_acrt_thread_detach 0000000180005c08 f   MSVCRT:ucrt_stubs.obj
 0001:00004c08       __scrt_stub_for_acrt_uninitialize 0000000180005c08 f   MSVCRT:ucrt_stubs.obj
 0001:00004c08       __scrt_stub_for_acrt_uninitialize_critical 0000000180005c08 f   MSVCRT:ucrt_stubs.obj
 0001:00004c08       __vcrt_initialize          0000000180005c08 f   MSVCRT:ucrt_stubs.obj
 0001:00004c08       __vcrt_thread_attach       0000000180005c08 f   MSVCRT:ucrt_stubs.obj
 0001:00004c08       __vcrt_thread_detach       0000000180005c08 f   MSVCRT:ucrt_stubs.obj
 0001:00004c08       __vcrt_uninitialize        0000000180005c08 f   MSVCRT:ucrt_stubs.obj
 0001:00004c08       __vcrt_uninitialize_critical 0000000180005c08 f   MSVCRT:ucrt_stubs.obj
 0001:00004c0c       __scrt_stub_for_is_c_termination_complete 0000000180005c0c f   MSVCRT:ucrt_stubs.obj
 0001:00004c0c       _is_c_termination_complete 0000000180005c0c f   MSVCRT:ucrt_stubs.obj
 0001:00004c20       _guard_dispatch_icall_nop  0000000180005c20 f   MSVCRT:guard_dispatch.obj
 0001:00004c40       _guard_xfg_dispatch_icall_nop 0000000180005c40 f   MSVCRT:guard_xfg_dispatch.obj
 0002:00000000       __imp_RtlCaptureContext    0000000180006000     kernel32:KERNEL32.dll
 0002:00000008       __imp_RtlLookupFunctionEntry 0000000180006008     kernel32:KERNEL32.dll
 0002:00000010       __imp_RtlVirtualUnwind     0000000180006010     kernel32:KERNEL32.dll
 0002:00000018       __imp_UnhandledExceptionFilter 0000000180006018     kernel32:KERNEL32.dll
 0002:00000020       __imp_SetUnhandledExceptionFilter 0000000180006020     kernel32:KERNEL32.dll
 0002:00000028       __imp_GetCurrentProcess    0000000180006028     kernel32:KERNEL32.dll
 0002:00000030       __imp_TerminateProcess     0000000180006030     kernel32:KERNEL32.dll
 0002:00000038       __imp_IsProcessorFeaturePresent 0000000180006038     kernel32:KERNEL32.dll
 0002:00000040       __imp_CloseHandle          0000000180006040     kernel32:KERNEL32.dll
 0002:00000048       __imp_InitializeCriticalSectionAndSpinCount 0000000180006048     kernel32:KERNEL32.dll
 0002:00000050       __imp_DeleteCriticalSection 0000000180006050     kernel32:KERNEL32.dll
 0002:00000058       __imp_CreateEventW         0000000180006058     kernel32:KERNEL32.dll
 0002:00000060       __imp_GetModuleHandleW     0000000180006060     kernel32:KERNEL32.dll
 0002:00000068       __imp_GetProcAddress       0000000180006068     kernel32:KERNEL32.dll
 0002:00000070       __imp_IsDebuggerPresent    0000000180006070     kernel32:KERNEL32.dll
 0002:00000078       __imp_QueryPerformanceCounter 0000000180006078     kernel32:KERNEL32.dll
 0002:00000080       __imp_GetCurrentProcessId  0000000180006080     kernel32:KERNEL32.dll
 0002:00000088       __imp_GetCurrentThreadId   0000000180006088     kernel32:KERNEL32.dll
 0002:00000090       __imp_GetSystemTimeAsFileTime 0000000180006090     kernel32:KERNEL32.dll
 0002:00000098       __imp_DisableThreadLibraryCalls 0000000180006098     kernel32:KERNEL32.dll
 0002:000000a0       __imp_InitializeSListHead  00000001800060a0     kernel32:KERNEL32.dll
 0002:000000a8       \177KERNEL32_NULL_THUNK_DATA 00000001800060a8     kernel32:KERNEL32.dll
 0002:000000b0       __imp_memcpy               00000001800060b0     vcruntime:VCRUNTIME140.dll
 0002:000000b8       __imp_memset               00000001800060b8     vcruntime:VCRUNTIME140.dll
 0002:000000c0       __imp_strchr               00000001800060c0     vcruntime:VCRUNTIME140.dll
 0002:000000c8       __imp___C_specific_handler 00000001800060c8     vcruntime:VCRUNTIME140.dll
 0002:000000d0       __imp___std_type_info_destroy_list 00000001800060d0     vcruntime:VCRUNTIME140.dll
 0002:000000d8       \177VCRUNTIME140_NULL_THUNK_DATA 00000001800060d8     vcruntime:VCRUNTIME140.dll
 0002:000000e0       __imp_strtol               00000001800060e0     ucrt:api-ms-win-crt-convert-l1-1-0.dll
 0002:000000e8       \177api-ms-win-crt-convert-l1-1-0_NULL_THUNK_DATA 00000001800060e8     ucrt:api-ms-win-crt-convert-l1-1-0.dll
 0002:000000f0       __imp_malloc               00000001800060f0     ucrt:api-ms-win-crt-heap-l1-1-0.dll
 0002:000000f8       __imp_free                 00000001800060f8     ucrt:api-ms-win-crt-heap-l1-1-0.dll
 0002:00000100       \177api-ms-win-crt-heap-l1-1-0_NULL_THUNK_DATA 0000000180006100     ucrt:api-ms-win-crt-heap-l1-1-0.dll
 0002:00000108       __imp__errno               0000000180006108     ucrt:api-ms-win-crt-runtime-l1-1-0.dll
 0002:00000110       __imp_exit                 0000000180006110     ucrt:api-ms-win-crt-runtime-l1-1-0.dll
 0002:00000118       __imp__cexit               0000000180006118     ucrt:api-ms-win-crt-runtime-l1-1-0.dll
 0002:00000120       __imp__crt_atexit          0000000180006120     ucrt:api-ms-win-crt-runtime-l1-1-0.dll
 0002:00000128       __imp__execute_onexit_table 0000000180006128     ucrt:api-ms-win-crt-runtime-l1-1-0.dll
 0002:00000130       __imp__register_onexit_function 0000000180006130     ucrt:api-ms-win-crt-runtime-l1-1-0.dll
 0002:00000138       __imp__initialize_onexit_table 0000000180006138     ucrt:api-ms-win-crt-runtime-l1-1-0.dll
 0002:00000140       __imp__initialize_narrow_environment 0000000180006140     ucrt:api-ms-win-crt-runtime-l1-1-0.dll
 0002:00000148       __imp__configure_narrow_argv 0000000180006148     ucrt:api-ms-win-crt-runtime-l1-1-0.dll
 0002:00000150       __imp__seh_filter_dll      0000000180006150     ucrt:api-ms-win-crt-runtime-l1-1-0.dll
 0002:00000158       __imp__initterm_e          0000000180006158     ucrt:api-ms-win-crt-runtime-l1-1-0.dll
 0002:00000160       __imp__initterm            0000000180006160     ucrt:api-ms-win-crt-runtime-l1-1-0.dll
 0002:00000168       \177api-ms-win-crt-runtime-l1-1-0_NULL_THUNK_DATA 0000000180006168     ucrt:api-ms-win-crt-runtime-l1-1-0.dll
 0002:00000170       __imp___acrt_iob_func      0000000180006170     ucrt:api-ms-win-crt-stdio-l1-1-0.dll
 0002:00000178       __imp_fflush               0000000180006178     ucrt:api-ms-win-crt-stdio-l1-1-0.dll
 0002:00000180       __imp___stdio_common_vsprintf 0000000180006180     ucrt:api-ms-win-crt-stdio-l1-1-0.dll
 0002:00000188       __imp___stdio_common_vfprintf 0000000180006188     ucrt:api-ms-win-crt-stdio-l1-1-0.dll
 0002:00000190       \177api-ms-win-crt-stdio-l1-1-0_NULL_THUNK_DATA 0000000180006190     ucrt:api-ms-win-crt-stdio-l1-1-0.dll
 0002:00000198       __imp_strcmp               0000000180006198     ucrt:api-ms-win-crt-string-l1-1-0.dll
 0002:000001a0       __imp__strdup              00000001800061a0     ucrt:api-ms-win-crt-string-l1-1-0.dll
 0002:000001a0       __imp_strdup               00000001800061a0     ucrt:api-ms-win-crt-string-l1-1-0.dll
 0002:000001a8       __imp_strlen               00000001800061a8     ucrt:api-ms-win-crt-string-l1-1-0.dll
 0002:000001b0       __imp_strpbrk              00000001800061b0     ucrt:api-ms-win-crt-string-l1-1-0.dll
 0002:000001b8       __imp_strncpy              00000001800061b8     ucrt:api-ms-win-crt-string-l1-1-0.dll
 0002:000001c0       \177api-ms-win-crt-string-l1-1-0_NULL_THUNK_DATA 00000001800061c0     ucrt:api-ms-win-crt-string-l1-1-0.dll
 0002:000001c8       __guard_check_icall_fptr   00000001800061c8     MSVCRT:guard_support.obj
 0002:000001d0       __guard_xfg_check_icall_fptr 00000001800061d0     MSVCRT:guard_support.obj
 0002:000001d8       __guard_dispatch_icall_fptr 00000001800061d8     MSVCRT:guard_support.obj
 0002:000001e0       __guard_xfg_dispatch_icall_fptr 00000001800061e0     MSVCRT:guard_support.obj
 0002:000001e8       __guard_xfg_table_dispatch_icall_fptr 00000001800061e8     MSVCRT:guard_support.obj
 0002:000001f0       __castguard_check_failure_os_handled_fptr 00000001800061f0     MSVCRT:guard_support.obj
 0002:000001f8       __guard_memcpy_fptr        00000001800061f8     vcruntime:softmemtag.obj
 0002:00000200       __xc_a                     0000000180006200     MSVCRT:initializers.obj
 0002:00000208       __xc_z                     0000000180006208     MSVCRT:initializers.obj
 0002:00000210       __xi_a                     0000000180006210     MSVCRT:initializers.obj
 0002:00000220       __xi_z                     0000000180006220     MSVCRT:initializers.obj
 0002:00000228       __xl_a                     0000000180006228     MSVCRT:tlssup.obj
 0002:00000230       __xl_z                     0000000180006230     MSVCRT:tlssup.obj
 0002:00000238       __xp_a                     0000000180006238     MSVCRT:initializers.obj
 0002:00000240       __xp_z                     0000000180006240     MSVCRT:initializers.obj
 0002:00000248       __xt_a                     0000000180006248     MSVCRT:initializers.obj
 0002:00000250       __xt_z                     0000000180006250     MSVCRT:initializers.obj
 0002:00000260       g_refKindStr               0000000180006260     libiterinstcls002.obj
 0002:00000410       ??_C@_09BPLDFGCI@unknown_0@ 0000000180006410     libiterinstcls002.obj
 0002:00000420       ??_C@_0BL@FPNMECJD@JVMTI_HEAP_REFERENCE_CLASS@ 0000000180006420     libiterinstcls002.obj
 0002:00000440       ??_C@_0BL@FKGKKLNM@JVMTI_HEAP_REFERENCE_FIELD@ 0000000180006440     libiterinstcls002.obj
 0002:00000460       ??_C@_0CD@CAEHCFJF@JVMTI_HEAP_REFERENCE_ARRAY_ELEM@ 0000000180006460     libiterinstcls002.obj
 0002:00000488       ??_C@_0CC@DNEBMCNK@JVMTI_HEAP_REFERENCE_CLASS_LOAD@ 0000000180006488     libiterinstcls002.obj
 0002:000004b0       ??_C@_0BN@CJMIPEBB@JVMTI_HEAP_REFERENCE_SIGNERS@ 00000001800064b0     libiterinstcls002.obj
 0002:000004d0       ??_C@_0CH@HBOIDPEB@JVMTI_HEAP_REFERENCE_PROTECTION@ 00000001800064d0     libiterinstcls002.obj
 0002:000004f8       ??_C@_0BP@MDKGDGKL@JVMTI_HEAP_REFERENCE_INTERFACE@ 00000001800064f8     libiterinstcls002.obj
 0002:00000518       ??_C@_0CC@JJMIHNJH@JVMTI_HEAP_REFERENCE_STATIC_FIE@ 0000000180006518     libiterinstcls002.obj
 0002:00000540       ??_C@_0CD@IDHEEGID@JVMTI_HEAP_REFERENCE_CONSTANT_P@ 0000000180006540     libiterinstcls002.obj
 0002:00000568       ??_C@_0CA@EFFCHNG@JVMTI_HEAP_REFERENCE_SUPERCLASS@ 0000000180006568     libiterinstcls002.obj
 0002:00000588       ??_C@_0L@PCDFHGCJ@unknown_11@ 0000000180006588     libiterinstcls002.obj
 0002:00000598       ??_C@_0L@NJBICFOK@unknown_12@ 0000000180006598     libiterinstcls002.obj
 0002:000005a8       ??_C@_0L@MAADBEKL@unknown_13@ 00000001800065a8     libiterinstcls002.obj
 0002:000005b8       ??_C@_0L@IPECICGM@unknown_14@ 00000001800065b8     libiterinstcls002.obj
 0002:000005c8       ??_C@_0L@JGFJLDCN@unknown_15@ 00000001800065c8     libiterinstcls002.obj
 0002:000005d8       ??_C@_0L@LNHEOAOO@unknown_16@ 00000001800065d8     libiterinstcls002.obj
 0002:000005e8       ??_C@_0L@KEGPNBKP@unknown_17@ 00000001800065e8     libiterinstcls002.obj
 0002:000005f8       ??_C@_0L@CDPHMNGA@unknown_18@ 00000001800065f8     libiterinstcls002.obj
 0002:00000608       ??_C@_0L@DKOMPMCB@unknown_19@ 0000000180006608     libiterinstcls002.obj
 0002:00000618       ??_C@_0L@OJGIPJDB@unknown_20@ 0000000180006618     libiterinstcls002.obj
 0002:00000628       ??_C@_0CA@KAOFNDEM@JVMTI_HEAP_REFERENCE_JNI_GLOBAL@ 0000000180006628     libiterinstcls002.obj
 0002:00000648       ??_C@_0CC@HPFAJBK@JVMTI_HEAP_REFERENCE_SYSTEM_CLA@ 0000000180006648     libiterinstcls002.obj
 0002:00000670       ??_C@_0BN@FDEGFOHC@JVMTI_HEAP_REFERENCE_MONITOR@ 0000000180006670     libiterinstcls002.obj
 0002:00000690       ??_C@_0CB@HKIBCMAJ@JVMTI_HEAP_REFERENCE_STACK_LOCA@ 0000000180006690     libiterinstcls002.obj
 0002:000006b8       ??_C@_0BP@EAACMMOE@JVMTI_HEAP_REFERENCE_JNI_LOCAL@ 00000001800066b8     libiterinstcls002.obj
 0002:000006d8       ??_C@_0BM@IJDEOGOE@JVMTI_HEAP_REFERENCE_THREAD@ 00000001800066d8     libiterinstcls002.obj
 0002:000006f8       ??_C@_0BL@EDGPPKC@JVMTI_HEAP_REFERENCE_OTHER@ 00000001800066f8     libiterinstcls002.obj
 0002:00000714       ??_C@_04BCJPDBDA@Code@     0000000180006714     libiterinstcls002.obj
 0002:00000720       ??_C@_0BA@OCLMCFKC@LineNumberTable@ 0000000180006720     libiterinstcls002.obj
 0002:00000730       ??_C@_0BD@CPAEPILC@LocalVariableTable@ 0000000180006730     libiterinstcls002.obj
 0002:00000748       ??_C@_0BH@NMBDNHBD@LocalVariableTypeTable@ 0000000180006748     libiterinstcls002.obj
 0002:00000760       ??_C@_0O@HIHEEDNJ@StackMapTable@ 0000000180006760     libiterinstcls002.obj
 0002:00000770       ??_C@_0L@HCDIAMJG@?9?5?$CFs?0?5?$CFd?3?5@ 0000000180006770     libiterinstcls002.obj
 0002:00000780       ??_C@_0JI@HLPECLFI@?$CD?5?4?4?4?6?$CD?5ERROR?3?5too?5many?5complai@ 0000000180006780     libiterinstcls002.obj
 0002:00000820       ??_C@_0ED@JNEKCCOB@The?5following?5fake?5exception?5st@ 0000000180006820     libiterinstcls002.obj
 0002:00000868       ??_C@_0CN@FCNMDFBH@nsk?4share?4Fake_Exception_for_RU@ 0000000180006868     libiterinstcls002.obj
 0002:00000898       ??_C@_08PGFFNAEI@?$CI?$CFs?3?$CFd?$CJ?5@ 0000000180006898     libiterinstcls002.obj
 0002:000008a8       ??_C@_0DP@IENMAEGI@s?2test?2hotspot?2jtreg?2vmTestbase@ 00000001800068a8     libiterinstcls002.obj
 0002:000008e8       ??_C@_0BL@NDJLFFJB@?7at?5nsk_lvcomplain?$CI?$CFs?3?$CFd?$CJ?6@ 00000001800068e8     libiterinstcls002.obj
 0002:00000908       ??_C@_0BC@JOOKAFKF@?$CD?5ERROR?3?5?$CFs?0?5?$CFd?3?5@ 0000000180006908     libiterinstcls002.obj
 0002:00000920       ??_C@_09KJEAHMEH@?$CD?5ERROR?3?5@ 0000000180006920     libiterinstcls002.obj
 0002:0000092c       ??_C@_02GPIOPFAK@?$DO?$DO@ 000000018000692c     libiterinstcls002.obj
 0002:00000930       ??_C@_02FODMEDOG@?$DM?$DM@ 0000000180006930     libiterinstcls002.obj
 0002:00000934       ??_C@_02DJGKEECL@?4?4@     0000000180006934     libiterinstcls002.obj
 0002:00000938       ??_C@_0O@CJPGJOAF@?9?5?$CFs?0?5?$CFd?3?5?$CFs?5@ 0000000180006938     libiterinstcls002.obj
 0002:00000948       ??_C@_0CB@IAKPDOIC@?$CD?5?5?5verified?5assertion?5is?5FALSE@ 0000000180006948     libiterinstcls002.obj
 0002:00000970       ??_C@_0CO@LGONDEPD@stdout?3?5fflush?5failed?5?9?5err?$DN?$CFd?5@ 0000000180006970     libiterinstcls002.obj
 0002:000009a0       ??_C@_0CO@KBGKJPBD@stderr?3?5fflush?5failed?5?9?5err?$DN?$CFd?5@ 00000001800069a0     libiterinstcls002.obj
 0002:000009d0       ??_C@_0BB@JCNMKLLK@JVMTI_ERROR_NONE@ 00000001800069d0     libiterinstcls002.obj
 0002:000009e8       ??_C@_0BL@LDIMKLPH@JVMTI_ERROR_INVALID_THREAD@ 00000001800069e8     libiterinstcls002.obj
 0002:00000a08       ??_C@_0CB@PJFPAIKJ@JVMTI_ERROR_INVALID_THREAD_GROU@ 0000000180006a08     libiterinstcls002.obj
 0002:00000a30       ??_C@_0BN@LLMKHMNF@JVMTI_ERROR_INVALID_PRIORITY@ 0000000180006a30     libiterinstcls002.obj
 0002:00000a50       ??_C@_0CB@MBOFKAGB@JVMTI_ERROR_THREAD_NOT_SUSPENDE@ 0000000180006a50     libiterinstcls002.obj
 0002:00000a78       ??_C@_0BN@FABOLPBI@JVMTI_ERROR_THREAD_SUSPENDED@ 0000000180006a78     libiterinstcls002.obj
 0002:00000a98       ??_C@_0BN@FDGNOBJM@JVMTI_ERROR_THREAD_NOT_ALIVE@ 0000000180006a98     libiterinstcls002.obj
 0002:00000ab8       ??_C@_0BL@GOBIFKNJ@JVMTI_ERROR_INVALID_OBJECT@ 0000000180006ab8     libiterinstcls002.obj
 0002:00000ad8       ??_C@_0BK@FCMAJPPC@JVMTI_ERROR_INVALID_CLASS@ 0000000180006ad8     libiterinstcls002.obj
 0002:00000af8       ??_C@_0BP@IKLLBKEB@JVMTI_ERROR_CLASS_NOT_PREPARED@ 0000000180006af8     libiterinstcls002.obj
 0002:00000b18       ??_C@_0BN@KLPPLKG@JVMTI_ERROR_INVALID_METHODID@ 0000000180006b18     libiterinstcls002.obj
 0002:00000b38       ??_C@_0BN@BCEKOKND@JVMTI_ERROR_INVALID_LOCATION@ 0000000180006b38     libiterinstcls002.obj
 0002:00000b58       ??_C@_0BM@DFDGPME@JVMTI_ERROR_INVALID_FIELDID@ 0000000180006b58     libiterinstcls002.obj
 0002:00000b78       ??_C@_0BL@NELIEPEC@JVMTI_ERROR_NO_MORE_FRAMES@ 0000000180006b78     libiterinstcls002.obj
 0002:00000b98       ??_C@_0BJ@BDBECFDM@JVMTI_ERROR_OPAQUE_FRAME@ 0000000180006b98     libiterinstcls002.obj
 0002:00000bb8       ??_C@_0BK@MIIFNLOB@JVMTI_ERROR_TYPE_MISMATCH@ 0000000180006bb8     libiterinstcls002.obj
 0002:00000bd8       ??_C@_0BJ@HPCAOILC@JVMTI_ERROR_INVALID_SLOT@ 0000000180006bd8     libiterinstcls002.obj
 0002:00000bf8       ??_C@_0BG@CHILOPNI@JVMTI_ERROR_DUPLICATE@ 0000000180006bf8     libiterinstcls002.obj
 0002:00000c10       ??_C@_0BG@DIEMLHKM@JVMTI_ERROR_NOT_FOUND@ 0000000180006c10     libiterinstcls002.obj
 0002:00000c28       ??_C@_0BM@NHMCKHOB@JVMTI_ERROR_INVALID_MONITOR@ 0000000180006c28     libiterinstcls002.obj
 0002:00000c48       ??_C@_0BO@PPEDAJGL@JVMTI_ERROR_NOT_MONITOR_OWNER@ 0000000180006c48     libiterinstcls002.obj
 0002:00000c68       ??_C@_0BG@FCAIPEID@JVMTI_ERROR_INTERRUPT@ 0000000180006c68     libiterinstcls002.obj
 0002:00000c80       ??_C@_0CB@EGDBNKOI@JVMTI_ERROR_INVALID_CLASS_FORMA@ 0000000180006c80     libiterinstcls002.obj
 0002:00000ca8       ??_C@_0CG@DGKOGIAL@JVMTI_ERROR_CIRCULAR_CLASS_DEFI@ 0000000180006ca8     libiterinstcls002.obj
 0002:00000cd0       ??_C@_0BP@ICEALPKC@JVMTI_ERROR_FAILS_VERIFICATION@ 0000000180006cd0     libiterinstcls002.obj
 0002:00000cf0       ??_C@_0DC@JDACLMIO@JVMTI_ERROR_UNSUPPORTED_REDEFIN@ 0000000180006cf0     libiterinstcls002.obj
 0002:00000d28       ??_C@_0DE@GKDKNOMJ@JVMTI_ERROR_UNSUPPORTED_REDEFIN@ 0000000180006d28     libiterinstcls002.obj
 0002:00000d60       ??_C@_0BO@LAFKIOG@JVMTI_ERROR_INVALID_TYPESTATE@ 0000000180006d60     libiterinstcls002.obj
 0002:00000d80       ??_C@_0DH@INDGCLLB@JVMTI_ERROR_UNSUPPORTED_REDEFIN@ 0000000180006d80     libiterinstcls002.obj
 0002:00000db8       ??_C@_0DE@NHEOMMGI@JVMTI_ERROR_UNSUPPORTED_REDEFIN@ 0000000180006db8     libiterinstcls002.obj
 0002:00000df0       ??_C@_0CA@EKPNJOEP@JVMTI_ERROR_UNSUPPORTED_VERSION@ 0000000180006df0     libiterinstcls002.obj
 0002:00000e10       ??_C@_0BN@OFFMAHHL@JVMTI_ERROR_NAMES_DONT_MATCH@ 0000000180006e10     libiterinstcls002.obj
 0002:00000e30       ??_C@_0DN@HHBBLAKE@JVMTI_ERROR_UNSUPPORTED_REDEFIN@ 0000000180006e30     libiterinstcls002.obj
 0002:00000e70       ??_C@_0DO@HMBGBGNA@JVMTI_ERROR_UNSUPPORTED_REDEFIN@ 0000000180006e70     libiterinstcls002.obj
 0002:00000eb0       ??_C@_0BP@PBECGKHJ@JVMTI_ERROR_UNMODIFIABLE_CLASS@ 0000000180006eb0     libiterinstcls002.obj
 0002:00000ed0       ??_C@_0BK@CANILEHF@JVMTI_ERROR_NOT_AVAILABLE@ 0000000180006ed0     libiterinstcls002.obj
 0002:00000ef0       ??_C@_0CE@INJKMEFK@JVMTI_ERROR_MUST_POSSESS_CAPABI@ 0000000180006ef0     libiterinstcls002.obj
 0002:00000f18       ??_C@_0BJ@LBFPFPDM@JVMTI_ERROR_NULL_POINTER@ 0000000180006f18     libiterinstcls002.obj
 0002:00000f38       ??_C@_0BP@CHJPNNEM@JVMTI_ERROR_ABSENT_INFORMATION@ 0000000180006f38     libiterinstcls002.obj
 0002:00000f58       ??_C@_0BP@OMFMNLC@JVMTI_ERROR_INVALID_EVENT_TYPE@ 0000000180006f58     libiterinstcls002.obj
 0002:00000f78       ??_C@_0BN@BIBNPHHO@JVMTI_ERROR_ILLEGAL_ARGUMENT@ 0000000180006f78     libiterinstcls002.obj
 0002:00000f98       ??_C@_0BK@KKNDHDCE@JVMTI_ERROR_NATIVE_METHOD@ 0000000180006f98     libiterinstcls002.obj
 0002:00000fb8       ??_C@_0BK@PMKCFHAE@JVMTI_ERROR_OUT_OF_MEMORY@ 0000000180006fb8     libiterinstcls002.obj
 0002:00000fd8       ??_C@_0BK@NNJBDMNB@JVMTI_ERROR_ACCESS_DENIED@ 0000000180006fd8     libiterinstcls002.obj
 0002:00000ff8       ??_C@_0BI@GHECLMNC@JVMTI_ERROR_WRONG_PHASE@ 0000000180006ff8     libiterinstcls002.obj
 0002:00001010       ??_C@_0BF@OLIHJOII@JVMTI_ERROR_INTERNAL@ 0000000180007010     libiterinstcls002.obj
 0002:00001028       ??_C@_0BO@EOHGKJHI@JVMTI_ERROR_UNATTACHED_THREAD@ 0000000180007028     libiterinstcls002.obj
 0002:00001048       ??_C@_0CA@LKHFDACL@JVMTI_ERROR_INVALID_ENVIRONMENT@ 0000000180007048     libiterinstcls002.obj
 0002:00001068       ??_C@_0BA@MMFHLOKK@?$DMunknown?5error?$DO@ 0000000180007068     libiterinstcls002.obj
 0002:00001078       ??_C@_0CF@CBHOKDB@throwable?5?$DN?5jni?9?$DOExceptionOccur@ 0000000180007078     libiterinstcls002.obj
 0002:000010a0       ??_C@_03OFAPEBGM@?$CFs?6@  00000001800070a0     libiterinstcls002.obj
 0002:000010a8       ??_C@_0DM@LPIGEGNJ@s?2test?2hotspot?2jtreg?2vmTestbase@ 00000001800070a8     libiterinstcls002.obj
 0002:000010e8       ??_C@_0CC@NFCNPEPK@Exception?5in?5JNI?5call?5?$CIcleared?$CJ@ 00000001800070e8     libiterinstcls002.obj
 0002:00001110       ??_C@_0BJ@IBAKFIKF@jni?9?$DOExceptionDescribe?$CI?$CJ@ 0000000180007110     libiterinstcls002.obj
 0002:00001130       ??_C@_0BG@GGKALKMH@jni?9?$DOExceptionClear?$CI?$CJ@ 0000000180007130     libiterinstcls002.obj
 0002:00001148       ??_C@_0CF@JMGFGJLJ@?$CD?5?5?5verified?5JNI?5assertion?5is?5F@ 0000000180007148     libiterinstcls002.obj
 0002:00001170       ??_C@_07KBAMPNJK@verbose@  0000000180007170     libiterinstcls002.obj
 0002:00001178       ??_C@_0DN@PKJBOLAP@nsk_jvmti_parseOptions?$CI?$CJ?3?5unexp@ 0000000180007178     libiterinstcls002.obj
 0002:000011b8       ??_C@_05IMBNNINJ@trace@    00000001800071b8     libiterinstcls002.obj
 0002:000011c0       ??_C@_0DD@BJKGNDMB@nsk_jvmti_parseOptions?$CI?$CJ?3?5no?5va@ 00000001800071c0     libiterinstcls002.obj
 0002:000011f4       ??_C@_04CGFJFPFD@none@     00000001800071f4     libiterinstcls002.obj
 0002:000011fc       ??_C@_06BMELKFMA@before@   00000001800071fc     libiterinstcls002.obj
 0002:00001204       ??_C@_05CMKPCFDK@after@    0000000180007204     libiterinstcls002.obj
 0002:0000120c       ??_C@_03NFKEKGGK@all@      000000018000720c     libiterinstcls002.obj
 0002:00001210       ??_C@_0DM@NDNJGJKE@nsk_jvmti_parseOptions?$CI?$CJ?3?5uexpe@ 0000000180007210     libiterinstcls002.obj
 0002:00001250       ??_C@_08NBBJKJO@waittime@  0000000180007250     libiterinstcls002.obj
 0002:00001260       ??_C@_0DO@CMHGAOHC@nsk_jvmti_parseOptions?$CI?$CJ?3?5not?5i@ 0000000180007260     libiterinstcls002.obj
 0002:000012a0       ??_C@_0DL@LNMPBDLN@nsk_jvmti_parseOptions?$CI?$CJ?3?5negat@ 00000001800072a0     libiterinstcls002.obj
 0002:000012e0       ??_C@_0DA@GMFJNOJH@nsk_jvmti_parseOptions?$CI?$CJ?3?5unkno@ 00000001800072e0     libiterinstcls002.obj
 0002:00001310       ??_C@_0CO@CCIAMEAN@nsk_jvmti_parseOptions?$CI?$CJ?3?5found@ 0000000180007310     libiterinstcls002.obj
 0002:00001340       ??_C@_0CJ@OEGPCGDL@nsk_jvmti_parseOptions?$CI?$CJ?3?5out?5o@ 0000000180007340     libiterinstcls002.obj
 0002:00001370       ??_C@_0DI@NMBHPGGF@nsk_jvmti_parseOptions?$CI?$CJ?3?5too?5m@ 0000000180007370     libiterinstcls002.obj
 0002:000013a8       ??_C@_03POGCGECB@?5?0?$HO@ 00000001800073a8     libiterinstcls002.obj
 0002:000013b0       ??_C@_0DC@GKLNPJIJ@nsk_jvmti_findOptionValue?$CI?$CJ?3?5op@ 00000001800073b0     libiterinstcls002.obj
 0002:000013e8       ??_C@_0DF@OPPIHBPJ@nsk_jvmti_findOptionIntValue?$CI?$CJ?3@ 00000001800073e8     libiterinstcls002.obj
 0002:00001420       ??_C@_0DO@DBKDODPI@nsk_jvmti_findOptionIntValue?$CI?$CJ?3@ 0000000180007420     libiterinstcls002.obj
 0002:00001460       ??_C@_0EE@NGNPKOJC@nsk_jvmti_findOptionIntValue?$CI?$CJ?3@ 0000000180007460     libiterinstcls002.obj
 0002:000014a8       ??_C@_0CB@MLNJNCLJ@?5?5jvmti?5error?3?5code?$DN?$CFd?0?5name?$DN?$CFs@ 00000001800074a8     libiterinstcls002.obj
 0002:000014d0       ??_C@_0CD@OHBGDKMK@?$CD?5?5?5jvmti?5error?3?5code?$DN?$CFd?0?5name?$DN@ 00000001800074d0     libiterinstcls002.obj
 0002:000014f8       ??_C@_0CG@JNNCGPHB@?$CD?5?5?5error?5expected?3?5code?$DN?$CFd?0?5na@ 00000001800074f8     libiterinstcls002.obj
 0002:00001520       ??_C@_0EB@IMGKPCGE@?$CIstr_obj?5?$DN?5jni?9?$DONewStringUTF?$CIco@ 0000000180007520     libiterinstcls002.obj
 0002:00001570       ??_C@_0EA@HFOGGBCC@s?2test?2hotspot?2jtreg?2vmTestbase@ 0000000180007570     libiterinstcls002.obj
 0002:000015b0       ??_C@_05KKCIMGE@error@     00000001800075b0     libiterinstcls002.obj
 0002:000015b8       ??_C@_0CJ@JACLEAA@Test?5failed?5by?5setFailStatus?$CI?$CJ?4@ 00000001800075b8     libiterinstcls002.obj
 0002:000015e8       ??_C@_0BD@HGNAOMCP@agent_data_monitor@ 00000001800075e8     libiterinstcls002.obj
 0002:00001600       ??_C@_0EB@OGCLGKLN@javaVM?9?$DOGetEnv?$CI?$CIvoid?5?$CK?$CK?$CJ?$CGjvmti_@ 0000000180007600     libiterinstcls002.obj
 0002:00001650       ??_C@_0EA@PNBCDMOA@s?2test?2hotspot?2jtreg?2vmTestbase@ 0000000180007650     libiterinstcls002.obj
 0002:00001690       ??_C@_0CI@DDPIFBGM@init_agent_data?$CIjvmti_env?0?5?$CGage@ 0000000180007690     libiterinstcls002.obj
 0002:000016b8       ??_C@_0DI@ILAHDLMP@?$CI?$CKagentThreadProc?$CJ?$CIjvmti_env?0?5a@ 00000001800076b8     libiterinstcls002.obj
 0002:000016f0       ??_C@_0BD@KDBALNLB@JVMTI?5agent?5thread@ 00000001800076f0     libiterinstcls002.obj
 0002:00001708       ??_C@_0BB@NOKBFPFO@java?1lang?1Thread@ 0000000180007708     libiterinstcls002.obj
 0002:0000171c       ??_C@_06FALKBLGB@?$DMinit?$DO@ 000000018000771c     libiterinstcls002.obj
 0002:00001728       ??_C@_0BG@IKDDPPGD@?$CILjava?1lang?1String?$DL?$CJV@ 0000000180007728     libiterinstcls002.obj
 0002:00001740       ??_C@_0EB@IFJBFEKC@?$CIthreadClass?5?$DN?5jni_env?9?$DOFindCla@ 0000000180007740     libiterinstcls002.obj
 0002:00001790       ??_C@_0GF@FGFIBKKL@?$CIthreadCtor?5?$DN?5jni_env?9?$DOGetMetho@ 0000000180007790     libiterinstcls002.obj
 0002:000017f8       ??_C@_0DN@NCPDJLOG@?$CIthreadName?5?$DN?5jni_env?9?$DONewStrin@ 00000001800077f8     libiterinstcls002.obj
 0002:00001840       ??_C@_0FE@PFKODBGC@?$CIthreadObject?5?$DN?5jni_env?9?$DONewObj@ 0000000180007840     libiterinstcls002.obj
 0002:000018a0       ??_C@_0ED@HOBAHHJI@?$CIthreadGlobalRef?5?$DN?5jni_env?9?$DONew@ 00000001800078a0     libiterinstcls002.obj
 0002:000018f0       ??_C@_0FN@HNJJAHFC@jvmti_env?9?$DORunAgentThread?$CIagent@ 00000001800078f0     libiterinstcls002.obj
 0002:00001950       ??_C@_0EA@MOJDNKDF@Debuggee?5status?5sync?5aborted?5be@ 0000000180007950     libiterinstcls002.obj
 0002:00001990       ??_C@_0CO@PGPGMHBJ@No?5status?5sync?5occured?5for?5time@ 0000000180007990     libiterinstcls002.obj
 0002:000019c0       ??_C@_0CL@DOEBDPKJ@Debuggee?5was?5not?5suspended?5on?5s@ 00000001800079c0     libiterinstcls002.obj
 0002:000019f0       ??_C@_0EA@EEOEJAEN@status?5?$DN?5syncDebuggeeStatus?$CIjni@ 00000001800079f0     libiterinstcls002.obj
 0002:00001a30       ??_C@_0BL@JBCFNBMB@nsk_jvmti_resetAgentData?$CI?$CJ@ 0000000180007a30     libiterinstcls002.obj
 0002:00001a50       ??_C@_0DN@NNGECJON@jvmti_env?9?$DOSetEventNotification@ 0000000180007a50     libiterinstcls002.obj
 0002:00001a90       ??_C@_0EL@LPBEELIP@s?2test?2hotspot?2jtreg?2vmTestbase@ 0000000180007a90     libiterinstcls002.obj
 0002:00001ae0       ??_C@_0CK@JDAMFDMJ@jvmti?9?$DOSetTag?$CIo?0?5tag?$CJ?5?$DN?$DN?5JVMTI_@ 0000000180007ae0     libiterinstcls002.obj
 0002:00001b10       ??_C@_0CC@DAMNHKNI@Can?8t?5set?5tag?5?$CFli?5for?5object?5?$CFl@ 0000000180007b10     libiterinstcls002.obj
 0002:00001b38       ??_C@_0DL@HAJPNKEF@jvmti?9?$DOGetObjectHashCode?$CIo?0?5?$CGha@ 0000000180007b38     libiterinstcls002.obj
 0002:00001b78       ??_C@_0BL@JFPIEOBF@Can?8t?5get?5hash?5object?5?$CFlx?6@ 0000000180007b78     libiterinstcls002.obj
 0002:00001b98       ??_C@_0BG@DICPHBKN@setTag?3?5?$CF08x?5?$DM?9?5?$CF?53li@ 0000000180007b98     libiterinstcls002.obj
 0002:00001bb0       ??_C@_0DH@FCEEBDMJ@?$CIs?5?$DN?5jni?9?$DOGetStringUTFChars?$CIsIn@ 0000000180007bb0     libiterinstcls002.obj
 0002:00001be8       ??_C@_0BJ@OKKGHDCN@Can?8t?5get?5string?5at?5?$CF?$CDp?6@ 0000000180007be8     libiterinstcls002.obj
 0002:00001c08       ??_C@_0BP@EKFLGGFJ@Can?8t?5get?5string?5at?5?$CF?$CDp?3?5null?6@ 0000000180007c08     libiterinstcls002.obj
 0002:00001c28       ??_C@_06ICODBHCL@?5?1?1?5?$CFs@ 0000000180007c28     libiterinstcls002.obj
 0002:00001c30       ??_C@_0DB@KGFPLEGO@?$CIr?5?$DN?5jvmti?9?$DOGetTag?$CIo?0?5?$CGtag?$CJ?$CJ?5?$DN?$DN@ 0000000180007c30     libiterinstcls002.obj
 0002:00001c68       ??_C@_0CO@PDAGBCGJ@Can?8t?5GetTag?5for?5object?5?$CFlx?4?5Re@ 0000000180007c68     libiterinstcls002.obj
 0002:00001c98       ??_C@_0CH@HPEODOHC@TEST_BUG?3?5Max?4?5number?5of?5refs?5r@ 0000000180007c98     libiterinstcls002.obj
 0002:00001cc0       ??_C@_0DI@PHFCABIM@?$CIr?5?$DN?5jvmti?9?$DOGetTag?$CIfrom?0?5?$CGtagFr@ 0000000180007cc0     libiterinstcls002.obj
 0002:00001cf8       ??_C@_0DI@MDEGFNKD@TEST_BUG?3?5Can?8t?5GetTag?5for?5obje@ 0000000180007cf8     libiterinstcls002.obj
 0002:00001d30       ??_C@_0DE@MLELJAHM@?$CIr?5?$DN?5jvmti?9?$DOGetTag?$CIto?0?5?$CGtagTo?$CJ?$CJ@ 0000000180007d30     libiterinstcls002.obj
 0002:00001d70       ??_C@_0EA@OLCLFBLL@?$CIobj?5?$DN?5jni?9?$DOGetObjectField?$CIfirs@ 0000000180007d70     libiterinstcls002.obj
 0002:00001db0       ??_C@_0GI@IGNNAHEC@s?2test?2hotspot?2jtreg?2vmTestbase@ 0000000180007db0     libiterinstcls002.obj
 0002:00001e18       ??_C@_0BL@HDOCIPLI@jvmti?9?$DOSetTag?$CIobj?0?5objTag?$CJ@ 0000000180007e18     libiterinstcls002.obj
 0002:00001e38       ??_C@_0BP@KLIOMM@?5?5?5?5?5?5?5?5tag?$DN?$CF?95ld?5object?$DN0x?$CFp?6@ 0000000180007e38     libiterinstcls002.obj
 0002:00001e58       ??_C@_0BJ@NBEMCAEP@jni?9?$DODeleteLocalRef?$CIobj?$CJ@ 0000000180007e58     libiterinstcls002.obj
 0002:00001e78       ??_C@_0CO@OFDFJEOH@Allocate?5memory?5for?5objects?5lis@ 0000000180007e78     libiterinstcls002.obj
 0002:00001eb0       ??_C@_0FH@KENAHJKN@jvmti?9?$DOAllocate?$CI?$CI?$CKobjectsCount?5@ 0000000180007eb0     libiterinstcls002.obj
 0002:00001f08       ??_C@_0BN@GHDOCCDB@?5?5?4?4?4?5allocated?5array?3?50x?$CFp?6@ 0000000180007f08     libiterinstcls002.obj
 0002:00001f28       ??_C@_0DF@OBOEEOG@nsk?1jvmti?1IterateOverInstancesO@ 0000000180007f28     libiterinstcls002.obj
 0002:00001f60       ??_C@_0BI@ENEOJHP@Find?5debugee?5class?3?5?$CFs?6@ 0000000180007f60     libiterinstcls002.obj
 0002:00001f78       ??_C@_0DP@MFMMLPOM@?$CIdebugeeClass?5?$DN?5jni?9?$DOFindClass?$CI@ 0000000180007f78     libiterinstcls002.obj
 0002:00001fb8       ??_C@_0BJ@DFGCANJI@?5?5?4?4?4?5found?5class?3?50x?$CFp?6@ 0000000180007fb8     libiterinstcls002.obj
 0002:00001fe0       ??_C@_0EE@GFMBJJDG@nsk?1jvmti?1IterateOverInstancesO@ 0000000180007fe0     libiterinstcls002.obj
 0002:00002028       ??_C@_0BM@GFHMIOD@Find?5root?5object?5class?3?5?$CFs?6@ 0000000180008028     libiterinstcls002.obj
 0002:00002050       ??_C@_0EG@LBKAPJFG@?$CIrootObjectClass?5?$DN?5jni?9?$DOFindCla@ 0000000180008050     libiterinstcls002.obj
 0002:000020a0       ??_C@_0EA@GEFFPKFJ@nsk?1jvmti?1IterateOverInstancesO@ 00000001800080a0     libiterinstcls002.obj
 0002:000020e0       ??_C@_0BN@JPFPOKGN@Find?5chain?5object?5class?3?5?$CFs?6@ 00000001800080e0     libiterinstcls002.obj
 0002:00002100       ??_C@_0EI@PFABFCAO@?$CIchainObjectClass?5?$DN?5jni?9?$DOFindCl@ 0000000180008100     libiterinstcls002.obj
 0002:00002148       ??_C@_0CJ@LICFCEOF@Create?5global?5ref?5to?5tested?5cla@ 0000000180008148     libiterinstcls002.obj
 0002:00002180       ??_C@_0EJ@OABJGKLK@?$CI?$CKtestedClass?5?$DN?5?$CIjclass?$CJ?5jni?9?$DON@ 0000000180008180     libiterinstcls002.obj
 0002:000021d0       ??_C@_0BI@DDGFIBLM@?5?5?4?4?4?5global?5ref?3?50x?$CFp?6@ 00000001800081d0     libiterinstcls002.obj
 0002:000021e8       ??_C@_06IEOJBDIK@object@   00000001800081e8     libiterinstcls002.obj
 0002:000021f0       ??_C@_0CI@IPDCJCKO@Find?5static?5field?5in?5debugee?5cl@ 00000001800081f0     libiterinstcls002.obj
 0002:00002220       ??_C@_0GJ@EJPDBEIJ@?$CIobjectField?5?$DN?5jni?9?$DOGetStaticFi@ 0000000180008220     libiterinstcls002.obj
 0002:00002290       ??_C@_0EG@FEGIKBDE@Lnsk?1jvmti?1IterateOverInstances@ 0000000180008290     libiterinstcls002.obj
 0002:000022d8       ??_C@_0BJ@MIIADDIH@?5?5?4?4?4?5got?5fieldID?3?50x?$CFp?6@ 00000001800082d8     libiterinstcls002.obj
 0002:000022f8       ??_C@_0P@OFCAMOEL@reachableChain@ 00000001800082f8     libiterinstcls002.obj
 0002:00002308       ??_C@_0CO@GJFDOONJ@Find?5instance?5field?5in?5root?5obj@ 0000000180008308     libiterinstcls002.obj
 0002:00002340       ??_C@_0HI@JPPGJND@?$CIreachableChainField?5?$DN?5jni?9?$DOGet@ 0000000180008340     libiterinstcls002.obj
 0002:000023c0       ??_C@_0EC@DMFJKFJP@Lnsk?1jvmti?1IterateOverInstances@ 00000001800083c0     libiterinstcls002.obj
 0002:00002408       ??_C@_0BB@HCMFGFMC@unreachableChain@ 0000000180008408     libiterinstcls002.obj
 0002:00002420       ??_C@_0HM@FNOMFGGD@?$CIunreachableChainField?5?$DN?5jni?9?$DOG@ 0000000180008420     libiterinstcls002.obj
 0002:0000249c       ??_C@_04DIFLAKIP@tail@     000000018000849c     libiterinstcls002.obj
 0002:000024a8       ??_C@_0CP@FJDMDHPJ@Find?5instance?5field?5in?5chain?5ob@ 00000001800084a8     libiterinstcls002.obj
 0002:000024e0       ??_C@_0GE@BFDKKHME@?$CItailField?5?$DN?5jni?9?$DOGetFieldID?$CIch@ 00000001800084e0     libiterinstcls002.obj
 0002:00002548       ??_C@_0CH@IEEMMCJA@Get?5root?5object?5from?5static?5fie@ 0000000180008548     libiterinstcls002.obj
 0002:00002570       ??_C@_0EP@FMMDHOMP@?$CIrootObject?5?$DN?5jni?9?$DOGetStaticObj@ 0000000180008570     libiterinstcls002.obj
 0002:000025c0       ??_C@_0BI@FNLCMIKO@?5?5?4?4?4?5got?5object?3?50x?$CFp?6@ 00000001800085c0     libiterinstcls002.obj
 0002:000025d8       ??_C@_0BP@MAGAMBHE@Obtain?5and?5tag?5chain?5objects?3?6@ 00000001800085d8     libiterinstcls002.obj
 0002:000025f8       ??_C@_0BK@PNAIFCCO@?5?5?5?5tested?5class?5object?3?6@ 00000001800085f8     libiterinstcls002.obj
 0002:00002618       ??_C@_0CM@LOOALEL@jvmti?9?$DOSetTag?$CI?$CKtestedClass?0?5tes@ 0000000180008618     libiterinstcls002.obj
 0002:00002648       ??_C@_0CJ@ELCOJLPK@?5?5?5?5reachable?5objects?5chain?3?5?$CFd@ 0000000180008648     libiterinstcls002.obj
 0002:00002678       ??_C@_0CL@LBFMJNLN@?5?5?5?5unreachable?5objects?5chain?3?5@ 0000000180008678     libiterinstcls002.obj
 0002:000026a8       ??_C@_0DC@ELMHCFIE@Following?5tagged?1untagged?5objec@ 00000001800086a8     libiterinstcls002.obj
 0002:000026e0       ??_C@_0BI@FLMBJNKJ@?5?5?5?5reachable?5objects?3?6@ 00000001800086e0     libiterinstcls002.obj
 0002:000026f8       ??_C@_0CF@JOOAJMNM@?5?5?5?5?5?5?5?5tag?$DN?$CF?95ld?5iterated?$DN?$CFd?5t@ 00000001800086f8     libiterinstcls002.obj
 0002:00002720       ??_C@_0FE@CNNPNBH@Reachable?5tagged?5object?5was?5not@ 0000000180008720     libiterinstcls002.obj
 0002:00002778       ??_C@_0BK@GHAJMINB@?5?5?5?5unreachable?5objects?3?6@ 0000000180008778     libiterinstcls002.obj
 0002:00002798       ??_C@_0DE@HDKIKJBP@?5?5?5?5?5?5?5?5tag?$DN?$CF?95ld?5iterated?$DN?$CF?93d@ 0000000180008798     libiterinstcls002.obj
 0002:000027d0       ??_C@_0GE@DHEFCCBM@Not?5collected?5unreachable?5tagge@ 00000001800087d0     libiterinstcls002.obj
 0002:00002838       ??_C@_0BH@NOGKHIJK@?5?5?5?5untagged?5objects?3?6@ 0000000180008838     libiterinstcls002.obj
 0002:00002850       ??_C@_0CI@LBNADMCD@?5?5?5?5?5?5?5?5total?$DN?$CF?93d?5iterated?$DN?$CFd?5@ 0000000180008850     libiterinstcls002.obj
 0002:00002880       ??_C@_0HB@NIJMLBJD@A?5number?5of?5untagged?5objects?5we@ 0000000180008880     libiterinstcls002.obj
 0002:000028f8       ??_C@_0DA@IABOOJJM@Release?5object?5reference?5to?5tes@ 00000001800088f8     libiterinstcls002.obj
 0002:00002928       ??_C@_0CC@JPMJEGPE@jni?9?$DODeleteGlobalRef?$CItestedClas@ 0000000180008928     libiterinstcls002.obj
 0002:00002950       ??_C@_0BP@JPEMGJLC@Deallocate?5objects?5list?3?50x?$CFp?6@ 0000000180008950     libiterinstcls002.obj
 0002:00002970       ??_C@_0DC@DFJJAFOM@jvmti?9?$DODeallocate?$CI?$CIunsigned?5cha@ 0000000180008970     libiterinstcls002.obj
 0002:000029b0       ??_C@_0EB@PKININME@?5?5heapObjectCallback?3?5class_tag@ 00000001800089b0     libiterinstcls002.obj
 0002:00002a00       ??_C@_0HM@MDOIAGKI@Unexpected?5class_tag?5passed?5to?5@ 0000000180008a00     libiterinstcls002.obj
 0002:00002a80       ??_C@_0HI@GDAEPDPH@null?5tag_ptr?5is?5passed?5to?5heapO@ 0000000180008a80     libiterinstcls002.obj
 0002:00002b00       ??_C@_0HH@EJCIHBIJ@Untagged?5object?5passed?5to?5heapO@ 0000000180008b00     libiterinstcls002.obj
 0002:00002b80       ??_C@_0HN@PJHHJHKA@Unknown?5tagged?5object?5passed?5to@ 0000000180008b80     libiterinstcls002.obj
 0002:00002c00       ??_C@_0GJ@KHPKLHCF@Unexpected?5user_data?5is?5passed?5@ 0000000180008c00     libiterinstcls002.obj
 0002:00002c70       ??_C@_0CB@KHPCBPAO@Wait?5for?5tested?5objects?5created@ 0000000180008c70     libiterinstcls002.obj
 0002:00002c98       ??_C@_0BP@LAIJOMPC@nsk_jvmti_waitForSync?$CItimeout?$CJ@ 0000000180008c98     libiterinstcls002.obj
 0002:00002cb8       ??_C@_0DG@CILGJCLA@?$DO?$DO?$DO?5Obtain?5and?5tag?5tested?5objec@ 0000000180008cb8     libiterinstcls002.obj
 0002:00002cf0       ??_C@_0FI@EOINHGJD@getTestedObjects?$CIjvmti?0?5jni?0?5ch@ 0000000180008cf0     libiterinstcls002.obj
 0002:00002d50       ??_C@_0FE@DOBPAFPL@?$DO?$DO?$DO?5Enable?5OBJECT_FREE?5event?5an@ 0000000180008d50     libiterinstcls002.obj
 0002:00002da8       ??_C@_0DJ@GDOKODHN@nsk_jvmti_enableEvents?$CIJVMTI_EN@ 0000000180008da8     libiterinstcls002.obj
 0002:00002de8       ??_C@_0BH@LECMGIIA@nsk_jvmti_resumeSync?$CI?$CJ@ 0000000180008de8     libiterinstcls002.obj
 0002:00002e00       ??_C@_0FB@NFNNGOBK@?$DO?$DO?$DO?5Iterate?5over?5instances?5of?5t@ 0000000180008e00     libiterinstcls002.obj
 0002:00002e60       ??_C@_0GN@EMDOMMCP@jvmti?9?$DOIterateOverInstancesOfCl@ 0000000180008e60     libiterinstcls002.obj
 0002:00002ed0       ??_C@_0EK@MHGOCBJB@?$DO?$DO?$DO?5Disable?5OBJECT_FREE?5event?5a@ 0000000180008ed0     libiterinstcls002.obj
 0002:00002f20       ??_C@_0DK@BBGCCCAH@nsk_jvmti_enableEvents?$CIJVMTI_DI@ 0000000180008f20     libiterinstcls002.obj
 0002:00002f60       ??_C@_0BF@MNKEFEOE@?$DO?$DO?$DO?5Clean?5used?5data?6@ 0000000180008f60     libiterinstcls002.obj
 0002:00002f80       ??_C@_0EL@OOAPAPIO@releaseTestedObjects?$CIjvmti?0?5jni@ 0000000180008f80     libiterinstcls002.obj
 0002:00002fd0       ??_C@_0BH@HPEOJMHL@Let?5debugee?5to?5finish?6@ 0000000180008fd0     libiterinstcls002.obj
 0002:00002fe8       ??_C@_0BL@ECKEAEGE@?5?5?$DMObjectFree?$DO?3?5tag?$DN?$CF?95ld?6@ 0000000180008fe8     libiterinstcls002.obj
 0002:00003008       ??_C@_0CA@MNKGCBCG@nsk_jvmti_parseOptions?$CIoptions?$CJ@ 0000000180009008     libiterinstcls002.obj
 0002:00003028       ??_C@_04NIDJFNBE@info@     0000000180009028     libiterinstcls002.obj
 0002:00003030       ??_C@_06DFFOHAMN@objref@   0000000180009030     libiterinstcls002.obj
 0002:00003038       ??_C@_08JAMFKCP@stackref@  0000000180009038     libiterinstcls002.obj
 0002:00003048       ??_C@_08KICKEILH@heaproot@ 0000000180009048     libiterinstcls002.obj
 0002:00003058       ??_C@_07MNCDLPNM@heapobj@  0000000180009058     libiterinstcls002.obj
 0002:00003060       ??_C@_0BP@PNAOMHNJ@Unknown?5option?5value?3?5info?$DN?$CFs?6@ 0000000180009060     libiterinstcls002.obj
 0002:00003080       ??_C@_07JPLKJBI@objects@   0000000180009080     libiterinstcls002.obj
 0002:00003088       ??_C@_0BA@LIAABLEG@chainLength?5?$DO?50@ 0000000180009088     libiterinstcls002.obj
 0002:00003098       ??_C@_0DN@MIAMNFPH@?$CIjvmti?5?$DN?5nsk_jvmti_createJVMTIE@ 0000000180009098     libiterinstcls002.obj
 0002:000030d8       ??_C@_0BO@DBKDIPGD@jvmti?9?$DOAddCapabilities?$CI?$CGcaps?$CJ@ 00000001800090d8     libiterinstcls002.obj
 0002:00003100       ??_C@_0EC@ODFGFOAJ@jvmti?9?$DOSetEventCallbacks?$CI?$CGevent@ 0000000180009100     libiterinstcls002.obj
 0002:00003148       ??_C@_0CL@PIACJIPK@nsk_jvmti_setAgentProc?$CIagentPro@ 0000000180009148     libiterinstcls002.obj
 0002:00003190       ??_C@_1EC@JIJBPKFM@?$AAa?$AAp?$AAi?$AA?9?$AAm?$AAs?$AA?9?$AAw?$AAi?$AAn?$AA?9?$AAc?$AAo?$AAr?$AAe@ 0000000180009190     MSVCRT:thread_safe_statics.obj
 0002:000031d8       ??_C@_1BK@MGMFAEKH@?$AAk?$AAe?$AAr?$AAn?$AAe?$AAl?$AA3?$AA2?$AA?4?$AAd?$AAl?$AAl@ 00000001800091d8     MSVCRT:thread_safe_statics.obj
 0002:000031f8       ??_C@_0BJ@JEBJOJFJ@SleepConditionVariableCS@ 00000001800091f8     MSVCRT:thread_safe_statics.obj
 0002:00003218       ??_C@_0BJ@PGPPEPCC@WakeAllConditionVariable@ 0000000180009218     MSVCRT:thread_safe_statics.obj
 0002:00003238       _pDefaultRawDllMain        0000000180009238     MSVCRT:dll_dllmain.obj
 0002:00003238       _pRawDllMain               0000000180009238     MSVCRT:dll_dllmain.obj
 0002:00003240       __xmm@ffffffffffffffffffffffffffffffff 0000000180009240     MSVCRT:utility.obj
 0002:00003250       _load_config_used          0000000180009250     MSVCRT:loadcfg.obj
 0002:00003400       _tls_used                  0000000180009400     MSVCRT:tlssup.obj
 0002:00003428       __volatile_metadata        0000000180009428     <linker-defined>
 0002:00003818       __rtc_iaa                  0000000180009818     MSVCRT:initsect.obj
 0002:00003820       __rtc_izz                  0000000180009820     MSVCRT:initsect.obj
 0002:00003828       __rtc_taa                  0000000180009828     MSVCRT:initsect.obj
 0002:00003830       __rtc_tzz                  0000000180009830     MSVCRT:initsect.obj
 0002:00003838       _tls_start                 0000000180009838     MSVCRT:tlssup.obj
 0002:0000383c       _Init_thread_epoch         000000018000983c     MSVCRT:thread_safe_statics.obj
 0002:00003840       _tls_end                   0000000180009840     MSVCRT:tlssup.obj
 0002:00003fb4       __IMPORT_DESCRIPTOR_KERNEL32 0000000180009fb4     kernel32:KERNEL32.dll
 0002:00003fc8       __IMPORT_DESCRIPTOR_VCRUNTIME140 0000000180009fc8     vcruntime:VCRUNTIME140.dll
 0002:00003fdc       __IMPORT_DESCRIPTOR_api-ms-win-crt-heap-l1-1-0 0000000180009fdc     ucrt:api-ms-win-crt-heap-l1-1-0.dll
 0002:00003ff0       __IMPORT_DESCRIPTOR_api-ms-win-crt-runtime-l1-1-0 0000000180009ff0     ucrt:api-ms-win-crt-runtime-l1-1-0.dll
 0002:00004004       __IMPORT_DESCRIPTOR_api-ms-win-crt-convert-l1-1-0 000000018000a004     ucrt:api-ms-win-crt-convert-l1-1-0.dll
 0002:00004018       __IMPORT_DESCRIPTOR_api-ms-win-crt-stdio-l1-1-0 000000018000a018     ucrt:api-ms-win-crt-stdio-l1-1-0.dll
 0002:0000402c       __IMPORT_DESCRIPTOR_api-ms-win-crt-string-l1-1-0 000000018000a02c     ucrt:api-ms-win-crt-string-l1-1-0.dll
 0002:00004040       __NULL_IMPORT_DESCRIPTOR   000000018000a040     kernel32:KERNEL32.dll
 0003:00000030       _Init_global_epoch         000000018000b030     MSVCRT:thread_safe_statics.obj
 0003:00000040       __security_cookie          000000018000b040     MSVCRT:gs_cookie.obj
 0003:00000048       __security_cookie_complement 000000018000b048     MSVCRT:gs_cookie.obj
 0003:00000050       __scrt_native_dllmain_reason 000000018000b050     MSVCRT:utility.obj
 0003:00000058       __isa_available            000000018000b058     MSVCRT:cpu_disp.obj
 0003:0000005c       __isa_enabled              000000018000b05c     MSVCRT:cpu_disp.obj
 0003:00000060       __memset_fast_string_threshold 000000018000b060     MSVCRT:cpu_disp.obj
 0003:00000068       __memset_nt_threshold      000000018000b068     MSVCRT:cpu_disp.obj
 0003:00000070       __scrt_ucrt_dll_is_in_use  000000018000b070     MSVCRT:ucrt_stubs.obj
 0003:00000080       g_wrongHeapCallbacks       000000018000b080     libiterinstcls002.obj
 0003:00000100       g_szTagInfo                000000018000b100     libiterinstcls002.obj
 0003:00002040       g_tagFlags                 000000018000d040     libiterinstcls002.obj
 0003:00002428       g_refsToVerifyCnt          000000018000d428     libiterinstcls002.obj
 0003:0000242c       g_fakeUserData             000000018000d42c     libiterinstcls002.obj
 0003:00002430       g_tagVisitCount            000000018000d430     libiterinstcls002.obj
 0003:000033d0       g_refsToVerify             000000018000e3d0     libiterinstcls002.obj
 0003:0001aad0       g_userDataError            0000000180025ad0     libiterinstcls002.obj
 0003:0001ac90       ?_OptionsStorage@?1??__local_stdio_printf_options@@9@4_KA 0000000180025c90     libiterinstcls002.obj
 0003:0001b258       _tls_index                 0000000180026258     MSVCRT:tlssup.obj
 0003:0001b260       __scrt_current_native_startup_state 0000000180026260     MSVCRT:utility.obj
 0003:0001b268       __scrt_native_startup_lock 0000000180026268     MSVCRT:utility.obj
 0003:0001b2a8       __scrt_debugger_hook_flag  00000001800262a8     MSVCRT:utility_desktop.obj
 0003:0001b2b0       ?__type_info_root_node@@3U__type_info_node@@A 00000001800262b0     MSVCRT:tncleanup.obj
 0003:0001b2c0       ?_OptionsStorage@?1??__local_stdio_scanf_options@@9@4_KA 00000001800262c0     MSVCRT:default_local_stdio_options.obj
 0003:0001b2c8       __favor                    00000001800262c8     MSVCRT:cpu_disp.obj
 0003:0001b2d0       __dyn_tls_init_callback    00000001800262d0     <common>

 entry point at        0001:00004330

 Static symbols

 0000:fffd7000       .debug$S                   0000000180000000     iterinstcls002.exp
 0000:fffd7000       .debug$S                   0000000180000000     vcruntime:VCRUNTIME140.dll
 0000:fffd7000       .debug$S                   0000000180000000     vcruntime:VCRUNTIME140.dll
 0000:fffd7000       .debug$S                   0000000180000000     vcruntime:VCRUNTIME140.dll
 0000:fffd7000       .debug$S                   0000000180000000     vcruntime:VCRUNTIME140.dll
 0000:fffd7000       .debug$S                   0000000180000000     vcruntime:VCRUNTIME140.dll
 0000:fffd7000       .debug$S                   0000000180000000     vcruntime:VCRUNTIME140.dll
 0000:fffd7000       .debug$S                   0000000180000000     vcruntime:VCRUNTIME140.dll
 0000:fffd7000       .debug$S                   0000000180000000     ucrt:api-ms-win-crt-convert-l1-1-0.dll
 0000:fffd7000       .debug$S                   0000000180000000     ucrt:api-ms-win-crt-heap-l1-1-0.dll
 0000:fffd7000       .debug$S                   0000000180000000     ucrt:api-ms-win-crt-heap-l1-1-0.dll
 0000:fffd7000       .debug$S                   0000000180000000     ucrt:api-ms-win-crt-heap-l1-1-0.dll
 0000:fffd7000       .debug$S                   0000000180000000     ucrt:api-ms-win-crt-heap-l1-1-0.dll
 0000:fffd7000       .debug$S                   0000000180000000     ucrt:api-ms-win-crt-runtime-l1-1-0.dll
 0000:fffd7000       .debug$S                   0000000180000000     ucrt:api-ms-win-crt-runtime-l1-1-0.dll
 0000:fffd7000       .debug$S                   0000000180000000     ucrt:api-ms-win-crt-runtime-l1-1-0.dll
 0000:fffd7000       .debug$S                   0000000180000000     ucrt:api-ms-win-crt-runtime-l1-1-0.dll
 0000:fffd7000       .debug$S                   0000000180000000     ucrt:api-ms-win-crt-runtime-l1-1-0.dll
 0000:fffd7000       .debug$S                   0000000180000000     ucrt:api-ms-win-crt-runtime-l1-1-0.dll
 0000:fffd7000       .debug$S                   0000000180000000     ucrt:api-ms-win-crt-runtime-l1-1-0.dll
 0000:fffd7000       .debug$S                   0000000180000000     ucrt:api-ms-win-crt-runtime-l1-1-0.dll
 0000:fffd7000       .debug$S                   0000000180000000     ucrt:api-ms-win-crt-runtime-l1-1-0.dll
 0000:fffd7000       .debug$S                   0000000180000000     ucrt:api-ms-win-crt-runtime-l1-1-0.dll
 0000:fffd7000       .debug$S                   0000000180000000     ucrt:api-ms-win-crt-runtime-l1-1-0.dll
 0000:fffd7000       .debug$S                   0000000180000000     ucrt:api-ms-win-crt-runtime-l1-1-0.dll
 0000:fffd7000       .debug$S                   0000000180000000     ucrt:api-ms-win-crt-runtime-l1-1-0.dll
 0000:fffd7000       .debug$S                   0000000180000000     ucrt:api-ms-win-crt-runtime-l1-1-0.dll
 0000:fffd7000       .debug$S                   0000000180000000     ucrt:api-ms-win-crt-runtime-l1-1-0.dll
 0000:fffd7000       .debug$S                   0000000180000000     ucrt:api-ms-win-crt-runtime-l1-1-0.dll
 0000:fffd7000       .debug$S                   0000000180000000     ucrt:api-ms-win-crt-stdio-l1-1-0.dll
 0000:fffd7000       .debug$S                   0000000180000000     ucrt:api-ms-win-crt-stdio-l1-1-0.dll
 0000:fffd7000       .debug$S                   0000000180000000     ucrt:api-ms-win-crt-stdio-l1-1-0.dll
 0000:fffd7000       .debug$S                   0000000180000000     ucrt:api-ms-win-crt-stdio-l1-1-0.dll
 0000:fffd7000       .debug$S                   0000000180000000     ucrt:api-ms-win-crt-stdio-l1-1-0.dll
 0000:fffd7000       .debug$S                   0000000180000000     ucrt:api-ms-win-crt-stdio-l1-1-0.dll
 0000:fffd7000       .debug$S                   0000000180000000     ucrt:api-ms-win-crt-stdio-l1-1-0.dll
 0000:fffd7000       .debug$S                   0000000180000000     ucrt:api-ms-win-crt-stdio-l1-1-0.dll
 0000:fffd7000       .debug$S                   0000000180000000     ucrt:api-ms-win-crt-stdio-l1-1-0.dll
 0000:fffd7000       .debug$S                   0000000180000000     ucrt:api-ms-win-crt-stdio-l1-1-0.dll
 0000:fffd7000       .debug$S                   0000000180000000     ucrt:api-ms-win-crt-string-l1-1-0.dll
 0000:fffd7000       .debug$S                   0000000180000000     ucrt:api-ms-win-crt-string-l1-1-0.dll
 0000:fffd7000       .debug$S                   0000000180000000     ucrt:api-ms-win-crt-string-l1-1-0.dll
 0000:fffd7000       .debug$S                   0000000180000000     ucrt:api-ms-win-crt-string-l1-1-0.dll
 0000:fffd7000       .debug$S                   0000000180000000     ucrt:api-ms-win-crt-string-l1-1-0.dll
 0000:fffd7000       .debug$S                   0000000180000000     ucrt:api-ms-win-crt-string-l1-1-0.dll
 0000:fffd7000       .debug$S                   0000000180000000     ucrt:api-ms-win-crt-string-l1-1-0.dll
 0000:fffd7000       .debug$S                   0000000180000000     ucrt:api-ms-win-crt-string-l1-1-0.dll
 0000:fffd7000       .debug$S                   0000000180000000     kernel32:KERNEL32.dll
 0000:fffd7000       .debug$S                   0000000180000000     kernel32:KERNEL32.dll
 0000:fffd7000       .debug$S                   0000000180000000     kernel32:KERNEL32.dll
 0000:fffd7000       .debug$S                   0000000180000000     kernel32:KERNEL32.dll
 0000:fffd7000       .debug$S                   0000000180000000     kernel32:KERNEL32.dll
 0000:fffd7000       .debug$S                   0000000180000000     kernel32:KERNEL32.dll
 0000:fffd7000       .debug$S                   0000000180000000     kernel32:KERNEL32.dll
 0000:fffd7000       .debug$S                   0000000180000000     kernel32:KERNEL32.dll
 0000:fffd7000       .debug$S                   0000000180000000     kernel32:KERNEL32.dll
 0000:fffd7000       .debug$S                   0000000180000000     kernel32:KERNEL32.dll
 0000:fffd7000       .debug$S                   0000000180000000     kernel32:KERNEL32.dll
 0000:fffd7000       .debug$S                   0000000180000000     kernel32:KERNEL32.dll
 0000:fffd7000       .debug$S                   0000000180000000     kernel32:KERNEL32.dll
 0000:fffd7000       .debug$S                   0000000180000000     kernel32:KERNEL32.dll
 0000:fffd7000       .debug$S                   0000000180000000     kernel32:KERNEL32.dll
 0000:fffd7000       .debug$S                   0000000180000000     kernel32:KERNEL32.dll
 0000:fffd7000       .debug$S                   0000000180000000     kernel32:KERNEL32.dll
 0000:fffd7000       .debug$S                   0000000180000000     kernel32:KERNEL32.dll
 0000:fffd7000       .debug$S                   0000000180000000     kernel32:KERNEL32.dll
 0000:fffd7000       .debug$S                   0000000180000000     kernel32:KERNEL32.dll
 0000:fffd7000       .debug$S                   0000000180000000     kernel32:KERNEL32.dll
 0000:fffd7000       .debug$S                   0000000180000000     kernel32:KERNEL32.dll
 0000:fffd7000       .debug$S                   0000000180000000     kernel32:KERNEL32.dll
 0000:fffd7000       .debug$S                   0000000180000000     kernel32:KERNEL32.dll
 0000:fffd7000       .debug$S                   0000000180000000     kernel32:KERNEL32.dll
 0000:fffd7000       .debug$S                   0000000180000000     kernel32:KERNEL32.dll
 0000:fffd7000       .debug$S                   0000000180000000     kernel32:KERNEL32.dll
 0000:fffd7000       .debug$S                   0000000180000000     kernel32:KERNEL32.dll
 0001:00001050       addRefToVerify             0000000180002050 f   libiterinstcls002.obj
 0001:000010bc       agentProc                  00000001800020bc f   libiterinstcls002.obj
 0001:00001500       agentThreadWrapper         0000000180002500 f   libiterinstcls002.obj
 0001:000016d8       checkTestedObjects         00000001800026d8 f   libiterinstcls002.obj
 0001:000018f8       check_option               00000001800028f8 f   libiterinstcls002.obj
 0001:00001b40       file_basename              0000000180002b40 f   libiterinstcls002.obj
 0001:00001bb4       getChainObjects            0000000180002bb4 f   libiterinstcls002.obj
 0001:00001e28       getTestedObjects           0000000180002e28 f   libiterinstcls002.obj
 0001:000036c0       releaseTestedObjects       00000001800046c0 f   libiterinstcls002.obj
 0001:00003810       startAgentThreadWrapper    0000000180004810 f   libiterinstcls002.obj
 0001:00003b50       syncDebuggeeStatus         0000000180004b50 f   libiterinstcls002.obj
 0001:00003df0       capture_previous_context   0000000180004df0 f   MSVCRT:gs_report.obj
 0001:00003e64       ?__scrt_initialize_thread_safe_statics@@YAHXZ 0000000180004e64 f   MSVCRT:thread_safe_statics.obj
 0001:00003f34       ?__scrt_uninitialize_thread_safe_statics@@YAXXZ 0000000180004f34 f   MSVCRT:thread_safe_statics.obj
 0001:00003fe0       $$000000                   0000000180004fe0     MSVCRT:amdsecgs.obj
 0001:00004010       ?dllmain_crt_dispatch@@YAHQEAUHINSTANCE__@@KQEAX@Z 0000000180005010 f   MSVCRT:dll_dllmain.obj
 0001:00004060       ?dllmain_crt_process_attach@@YAHQEAUHINSTANCE__@@QEAX@Z 0000000180005060 f   MSVCRT:dll_dllmain.obj
 0001:00004178       ?dllmain_crt_process_detach@@YAH_N@Z 0000000180005178 f   MSVCRT:dll_dllmain.obj
 0001:000041fc       ?dllmain_dispatch@@YAHQEAUHINSTANCE__@@KQEAX@Z 00000001800051fc f   MSVCRT:dll_dllmain.obj
 0001:00004c10       $$000000                   0000000180005c10     MSVCRT:guard_dispatch.obj
 0001:00004c30       $$000000                   0000000180005c30     MSVCRT:guard_xfg_dispatch.obj
 0001:00004c46       ?fin$0@?0??dllmain_crt_process_attach@@YAHQEAUHINSTANCE__@@QEAX@Z@4HA 0000000180005c46 f   MSVCRT:dll_dllmain.obj
 0001:00004c5d       ?fin$0@?0??dllmain_crt_process_detach@@YAH_N@Z@4HA 0000000180005c5d f   MSVCRT:dll_dllmain.obj
 0001:00004c76       ?fin$1@?0??dllmain_crt_process_detach@@YAH_N@Z@4HA 0000000180005c76 f   MSVCRT:dll_dllmain.obj
 0001:00004c8a       ?filt$0@?0??dllmain_dispatch@@YAHQEAUHINSTANCE__@@KQEAX@Z@4HA 0000000180005c8a f   MSVCRT:dll_dllmain.obj
 0001:00004cc0       __scrt_is_nonwritable_in_current_image$filt$0 0000000180005cc0 f   MSVCRT:utility.obj
 0002:00000218       ?__scrt_initialize_tss_var@@3P6AHXZEA 0000000180006218     MSVCRT:thread_safe_statics.obj
 0002:00000340       ?opcLengths@@3QBEB         0000000180006340     libiterinstcls002.obj
 0002:00003178       GS_ExceptionPointers       0000000180009178     MSVCRT:gs_report.obj
 0002:00003848       $unwind$fprintf            0000000180009848     libiterinstcls002.obj
 0002:00003854       $unwind$printf             0000000180009854     libiterinstcls002.obj
 0002:00003860       $unwind$?NewObject@JNIEnv_@@QEAAPEAV_jobject@@PEAV_jclass@@PEAU_jmethodID@@ZZ 0000000180009860     libiterinstcls002.obj
 0002:00003860       $unwind$nsk_lcomplain      0000000180009860     libiterinstcls002.obj
 0002:00003860       $unwind$nsk_ldisplay       0000000180009860     libiterinstcls002.obj
 0002:00003868       $unwind$nsk_jvmti_waitForSync 0000000180009868     libiterinstcls002.obj
 0002:00003868       $unwind$nsk_lvdisplay      0000000180009868     libiterinstcls002.obj
 0002:00003868       $unwind$_RTC_Initialize    0000000180009868     MSVCRT:initsect.obj
 0002:00003868       $unwind$_RTC_Terminate     0000000180009868     MSVCRT:initsect.obj
 0002:00003868       $unwind$?__scrt_initialize_thread_safe_statics@@YAHXZ 0000000180009868     MSVCRT:thread_safe_statics.obj
 0002:00003874       $unwind$nsk_complain       0000000180009874     libiterinstcls002.obj
 0002:00003874       $unwind$nsk_printf         0000000180009874     libiterinstcls002.obj
 0002:0000387c       $unwind$nsk_lvcomplain     000000018000987c     libiterinstcls002.obj
 0002:00003894       $unwind$nsk_ltrace         0000000180009894     libiterinstcls002.obj
 0002:00003894       $unwind$__report_gsfailure 0000000180009894     MSVCRT:gs_report.obj
 0002:0000389c       $unwind$callbackObjectFree 000000018000989c     libiterinstcls002.obj
 0002:0000389c       $unwind$nsk_lvtrace        000000018000989c     libiterinstcls002.obj
 0002:0000389c       $unwind$__raise_securityfailure 000000018000989c     MSVCRT:gs_report.obj
 0002:0000389c       $unwind$__scrt_initialize_crt 000000018000989c     MSVCRT:utility.obj
 0002:0000389c       $unwind$__scrt_initialize_onexit_tables 000000018000989c     MSVCRT:utility.obj
 0002:0000389c       $unwind$__scrt_release_startup_lock 000000018000989c     MSVCRT:utility.obj
 0002:0000389c       $unwind$__scrt_uninitialize_crt 000000018000989c     MSVCRT:utility.obj
 0002:0000389c       $unwind$_onexit            000000018000989c     MSVCRT:utility.obj
 0002:000038a4       $unwind$nsk_lverify        00000001800098a4     libiterinstcls002.obj
 0002:000038b4       $unwind$nsk_vprintf        00000001800098b4     libiterinstcls002.obj
 0002:000038c4       $unwind$?nsk_jni_lverify@@YAHHPEAUJNIEnv_@@HQEBDH1ZZ 00000001800098c4     libiterinstcls002.obj
 0002:000038d8       $unwind$?nsk_jni_check_exception@@YAHPEAUJNIEnv_@@QEBDH@Z 00000001800098d8     libiterinstcls002.obj
 0002:000038f4       $unwind$nsk_jvmti_parseOptions 00000001800098f4     libiterinstcls002.obj
 0002:00003910       $unwind$nsk_jvmti_createJVMTIEnv 0000000180009910     libiterinstcls002.obj
 0002:00003924       $unwind$Java_nsk_jvmti_unit_FollowReferences_FollowRefObjects_resetTags 0000000180009924     libiterinstcls002.obj
 0002:00003924       $unwind$addRefToVerify     0000000180009924     libiterinstcls002.obj
 0002:00003924       $unwind$nsk_jvmti_resetAgentData 0000000180009924     libiterinstcls002.obj
 0002:00003924       $unwind$nsk_jvmti_resumeSync 0000000180009924     libiterinstcls002.obj
 0002:00003924       $unwind$nsk_jvmti_setFailStatus 0000000180009924     libiterinstcls002.obj
 0002:00003924       $unwind$__scrt_initialize_default_local_stdio_options 0000000180009924     MSVCRT:default_local_stdio_options.obj
 0002:00003924       $unwind$?dllmain_crt_dispatch@@YAHQEAUHINSTANCE__@@KQEAX@Z 0000000180009924     MSVCRT:dll_dllmain.obj
 0002:00003924       $unwind$DllMain            0000000180009924     MSVCRT:dll_dllmain_stub.obj
 0002:00003924       $unwind$__GSHandlerCheck   0000000180009924     MSVCRT:gshandler.obj
 0002:00003924       $unwind$?__scrt_uninitialize_thread_safe_statics@@YAXXZ 0000000180009924     MSVCRT:thread_safe_statics.obj
 0002:00003924       $unwind$__scrt_acquire_startup_lock 0000000180009924     MSVCRT:utility.obj
 0002:00003924       $unwind$__scrt_dllmain_after_initialize_c 0000000180009924     MSVCRT:utility.obj
 0002:00003924       $unwind$__scrt_dllmain_before_initialize_c 0000000180009924     MSVCRT:utility.obj
 0002:00003924       $unwind$__scrt_dllmain_crt_thread_attach 0000000180009924     MSVCRT:utility.obj
 0002:00003924       $unwind$__scrt_dllmain_crt_thread_detach 0000000180009924     MSVCRT:utility.obj
 0002:00003924       $unwind$__scrt_dllmain_uninitialize_c 0000000180009924     MSVCRT:utility.obj
 0002:00003924       $unwind$__scrt_dllmain_uninitialize_critical 0000000180009924     MSVCRT:utility.obj
 0002:00003924       $unwind$atexit             0000000180009924     MSVCRT:utility.obj
 0002:0000392c       $unwind$nsk_jvmti_enableEvents 000000018000992c     libiterinstcls002.obj
 0002:00003944       $unwind$check_option       0000000180009944     libiterinstcls002.obj
 0002:00003944       $unwind$nsk_jvmti_findOptionValue 0000000180009944     libiterinstcls002.obj
 0002:00003944       $unwind$_DllMainCRTStartup 0000000180009944     MSVCRT:dll_dllmain.obj
 0002:00003954       $unwind$nsk_jvmti_findOptionIntValue 0000000180009954     libiterinstcls002.obj
 0002:00003964       $unwind$nsk_jvmti_lverify  0000000180009964     libiterinstcls002.obj
 0002:00003978       $unwind$exitOnError        0000000180009978     libiterinstcls002.obj
 0002:00003988       $unwind$Java_nsk_share_jvmti_ArgumentHandler_getAgentOptionsString 0000000180009988     libiterinstcls002.obj
 0002:0000399c       $unwind$Java_nsk_jvmti_unit_FollowReferences_FollowRefObjects_getTag 000000018000999c     libiterinstcls002.obj
 0002:0000399c       $unwind$Java_nsk_share_jvmti_DebugeeClass_checkStatus 000000018000999c     libiterinstcls002.obj
 0002:0000399c       $unwind$agentThreadWrapper 000000018000999c     libiterinstcls002.obj
 0002:000039ac       $unwind$startAgentThreadWrapper 00000001800099ac     libiterinstcls002.obj
 0002:000039c8       $unwind$syncDebuggeeStatus 00000001800099c8     libiterinstcls002.obj
 0002:000039c8       $unwind$__scrt_dllmain_exception_filter 00000001800099c8     MSVCRT:utility.obj
 0002:000039dc       $unwind$Java_nsk_share_jvmti_DebugeeClass_resetAgentData 00000001800099dc     libiterinstcls002.obj
 0002:000039e4       $unwind$MA_checkStatus     00000001800099e4     libiterinstcls002.obj
 0002:000039f8       $unwind$Java_nsk_jvmti_unit_FollowReferences_FollowRefObjects_setTag 00000001800099f8     libiterinstcls002.obj
 0002:00003a10       $unwind$Java_nsk_jvmti_unit_FollowReferences_FollowRefObjects_addRefToVerify 0000000180009a10     libiterinstcls002.obj
 0002:00003a2c       $unwind$Agent_Initialize   0000000180009a2c     libiterinstcls002.obj
 0002:00003a4c       $unwind$getChainObjects    0000000180009a4c     libiterinstcls002.obj
 0002:00003a68       $unwind$getTestedObjects   0000000180009a68     libiterinstcls002.obj
 0002:00003a80       $unwind$checkTestedObjects 0000000180009a80     libiterinstcls002.obj
 0002:00003a9c       $unwind$releaseTestedObjects 0000000180009a9c     libiterinstcls002.obj
 0002:00003ab4       $unwind$heapObjectCallback 0000000180009ab4     libiterinstcls002.obj
 0002:00003acc       $unwind$agentProc          0000000180009acc     libiterinstcls002.obj
 0002:00003ae8       $unwind$capture_previous_context 0000000180009ae8     MSVCRT:gs_report.obj
 0002:00003af4       $unwind$__GSHandlerCheckCommon 0000000180009af4     MSVCRT:gshandler.obj
 0002:00003b00       $xdatasym                  0000000180009b00     MSVCRT:amdsecgs.obj
 0002:00003b04       $unwind$?dllmain_crt_process_attach@@YAHQEAUHINSTANCE__@@QEAX@Z 0000000180009b04     MSVCRT:dll_dllmain.obj
 0002:00003b40       $unwind$?fin$0@?0??dllmain_crt_process_attach@@YAHQEAUHINSTANCE__@@QEAX@Z@4HA 0000000180009b40     MSVCRT:dll_dllmain.obj
 0002:00003b40       $unwind$?fin$0@?0??dllmain_crt_process_detach@@YAH_N@Z@4HA 0000000180009b40     MSVCRT:dll_dllmain.obj
 0002:00003b40       $unwind$?fin$1@?0??dllmain_crt_process_detach@@YAH_N@Z@4HA 0000000180009b40     MSVCRT:dll_dllmain.obj
 0002:00003b48       $unwind$?dllmain_crt_process_detach@@YAH_N@Z 0000000180009b48     MSVCRT:dll_dllmain.obj
 0002:00003b9c       $unwind$?dllmain_dispatch@@YAHQEAUHINSTANCE__@@KQEAX@Z 0000000180009b9c     MSVCRT:dll_dllmain.obj
 0002:00003bc4       $unwind$?filt$0@?0??dllmain_dispatch@@YAHQEAUHINSTANCE__@@KQEAX@Z@4HA 0000000180009bc4     MSVCRT:dll_dllmain.obj
 0002:00003bcc       $unwind$__scrt_is_nonwritable_in_current_image 0000000180009bcc     MSVCRT:utility.obj
 0002:00003bec       $unwind$__scrt_is_nonwritable_in_current_image$filt$0 0000000180009bec     MSVCRT:utility.obj
 0002:00003bf4       $unwind$__scrt_fastfail    0000000180009bf4     MSVCRT:utility_desktop.obj
 0002:00003c04       $unwind$__security_init_cookie 0000000180009c04     MSVCRT:gs_support.obj
 0002:00003c10       $unwind$__isa_available_init 0000000180009c10     MSVCRT:cpu_disp.obj
 0002:00003c20       $xdatasym                  0000000180009c20     MSVCRT:guard_dispatch.obj
 0002:00003c28       $xdatasym                  0000000180009c28     MSVCRT:guard_xfg_dispatch.obj
 0002:00003c30       .edata                     0000000180009c30     iterinstcls002.exp
 0002:00003c58       rgpv                       0000000180009c58     iterinstcls002.exp
 0002:00003c94       rgszName                   0000000180009c94     iterinstcls002.exp
 0002:00003cd0       rgwOrd                     0000000180009cd0     iterinstcls002.exp
 0002:00003cee       szName                     0000000180009cee     iterinstcls002.exp
 0002:00003d01       $N00001                    0000000180009d01     iterinstcls002.exp
 0002:00003d10       $N00002                    0000000180009d10     iterinstcls002.exp
 0002:00003d1d       $N00003                    0000000180009d1d     iterinstcls002.exp
 0002:00003d62       $N00004                    0000000180009d62     iterinstcls002.exp
 0002:00003d9f       $N00005                    0000000180009d9f     iterinstcls002.exp
 0002:00003de7       $N00006                    0000000180009de7     iterinstcls002.exp
 0002:00003e27       $N00007                    0000000180009e27     iterinstcls002.exp
 0002:00003e64       $N00008                    0000000180009e64     iterinstcls002.exp
 0002:00003e9f       $N00009                    0000000180009e9f     iterinstcls002.exp
 0002:00003ecd       $N00010                    0000000180009ecd     iterinstcls002.exp
 0002:00003efe       $N00011                    0000000180009efe     iterinstcls002.exp
 0002:00003f2d       $N00012                    0000000180009f2d     iterinstcls002.exp
 0002:00003f5c       $N00013                    0000000180009f5c     iterinstcls002.exp
 0002:00003f91       $N00014                    0000000180009f91     iterinstcls002.exp
 0002:00003fa0       $N00015                    0000000180009fa0     iterinstcls002.exp
 0002:0000440a       .idata$6                   000000018000a40a     kernel32:KERNEL32.dll
 0002:0000446e       .idata$6                   000000018000a46e     vcruntime:VCRUNTIME140.dll
 0002:00004600       .idata$6                   000000018000a600     ucrt:api-ms-win-crt-heap-l1-1-0.dll
 0002:00004620       .idata$6                   000000018000a620     ucrt:api-ms-win-crt-runtime-l1-1-0.dll
 0002:00004642       .idata$6                   000000018000a642     ucrt:api-ms-win-crt-convert-l1-1-0.dll
 0002:00004664       .idata$6                   000000018000a664     ucrt:api-ms-win-crt-stdio-l1-1-0.dll
 0002:00004684       .idata$6                   000000018000a684     ucrt:api-ms-win-crt-string-l1-1-0.dll
 0003:00000000       ?codeAttributeName@@3PEBDEB 000000018000b000     libiterinstcls002.obj
 0003:00000008       ?lineNumberAttributeName@@3PEBDEB 000000018000b008     libiterinstcls002.obj
 0003:00000010       ?localVarAttributeName@@3PEBDEB 000000018000b010     libiterinstcls002.obj
 0003:00000018       ?localVarTypeAttributeName@@3PEBDEB 000000018000b018     libiterinstcls002.obj
 0003:00000020       ?stackMapAttributeName@@3PEBDEB 000000018000b020     libiterinstcls002.obj
 0003:00000028       ?callBytes@@3PAEA          000000018000b028     libiterinstcls002.obj
 0003:0000002c       ?allocBytes@@3PAEA         000000018000b02c     libiterinstcls002.obj
 0003:0001aad4       redefineAttempted          0000000180025ad4     libiterinstcls002.obj
 0003:0001aad8       nsk_context                0000000180025ad8     libiterinstcls002.obj
 0003:0001aae4       redefineSucceed            0000000180025ae4     libiterinstcls002.obj
 0003:0001aae8       agentFailed                0000000180025ae8     libiterinstcls002.obj
 0003:0001aaec       currentAgentStatus         0000000180025aec     libiterinstcls002.obj
 0003:0001aaf0       context                    0000000180025af0     libiterinstcls002.obj
 0003:0001aba8       agentThread                0000000180025ba8     libiterinstcls002.obj
 0003:0001abb0       agentThreadProc            0000000180025bb0     libiterinstcls002.obj
 0003:0001abb8       agentThreadArg             0000000180025bb8     libiterinstcls002.obj
 0003:0001abc0       agent_data                 0000000180025bc0     libiterinstcls002.obj
 0003:0001abd0       jvmti_env                  0000000180025bd0     libiterinstcls002.obj
 0003:0001abd8       jvm                        0000000180025bd8     libiterinstcls002.obj
 0003:0001abe0       jni_env                    0000000180025be0     libiterinstcls002.obj
 0003:0001abe8       checkStatus_func           0000000180025be8     libiterinstcls002.obj
 0003:0001abf0       ?codeAttributeIndex@@3GA   0000000180025bf0     libiterinstcls002.obj
 0003:0001abf4       ?lineNumberAttributeIndex@@3GA 0000000180025bf4     libiterinstcls002.obj
 0003:0001abf8       ?localVarAttributeIndex@@3GA 0000000180025bf8     libiterinstcls002.obj
 0003:0001abfc       ?localVarTypeAttributeIndex@@3GA 0000000180025bfc     libiterinstcls002.obj
 0003:0001ac00       ?stackMapAttributeIndex@@3GA 0000000180025c00     libiterinstcls002.obj
 0003:0001ac04       ?stackFrameOffset@@3GA     0000000180025c04     libiterinstcls002.obj
 0003:0001ac08       ?mode@@3HA                 0000000180025c08     libiterinstcls002.obj
 0003:0001ac0c       ?constantPoolSize@@3GA     0000000180025c0c     libiterinstcls002.obj
 0003:0001ac10       ?orig@@3PEBEEB             0000000180025c10     libiterinstcls002.obj
 0003:0001ac18       ?gen@@3PEAEEA              0000000180025c18     libiterinstcls002.obj
 0003:0001ac20       ?inputPos@@3PEAEEA         0000000180025c20     libiterinstcls002.obj
 0003:0001ac28       ?endPos@@3PEBEEB           0000000180025c28     libiterinstcls002.obj
 0003:0001ac30       ?genPos@@3PEAEEA           0000000180025c30     libiterinstcls002.obj
 0003:0001ac38       ?markPos@@3PEAEEA          0000000180025c38     libiterinstcls002.obj
 0003:0001ac40       ?constantPool@@3PEAPEADEA  0000000180025c40     libiterinstcls002.obj
 0003:0001ac48       ?constantPoolCount@@3GA    0000000180025c48     libiterinstcls002.obj
 0003:0001ac4c       ?zeroBytes@@3PAEA          0000000180025c4c     libiterinstcls002.obj
 0003:0001ac50       ?codeLength@@3IA           0000000180025c50     libiterinstcls002.obj
 0003:0001ac54       info                       0000000180025c54     libiterinstcls002.obj
 0003:0001ac58       ?map@@3PEAIEA              0000000180025c58     libiterinstcls002.obj
 0003:0001ac60       ?widening@@3PEACEA         0000000180025c60     libiterinstcls002.obj
 0003:0001ac68       timeout                    0000000180025c68     libiterinstcls002.obj
 0003:0001ac70       chainLength                0000000180025c70     libiterinstcls002.obj
 0003:0001ac74       objectsCount               0000000180025c74     libiterinstcls002.obj
 0003:0001ac78       objectDescList             0000000180025c78     libiterinstcls002.obj
 0003:0001ac80       foundUntagged              0000000180025c80     libiterinstcls002.obj
 0003:0001ac84       fakeUserData               0000000180025c84     libiterinstcls002.obj
 0003:0001ac88       userDataError              0000000180025c88     libiterinstcls002.obj
 0003:0001aca0       GS_ExceptionRecord         0000000180025ca0     MSVCRT:gs_report.obj
 0003:0001ad40       GS_ContextRecord           0000000180025d40     MSVCRT:gs_report.obj
 0003:0001b210       ?g_tss_cv@@3U_RTL_CONDITION_VARIABLE@@A 0000000180026210     MSVCRT:thread_safe_statics.obj
 0003:0001b218       ?g_tss_event@@3PEAXEA      0000000180026218     MSVCRT:thread_safe_statics.obj
 0003:0001b220       ?g_tss_mutex@@3U_RTL_CRITICAL_SECTION@@A 0000000180026220     MSVCRT:thread_safe_statics.obj
 0003:0001b248       ?g_sleep_condition_variable_cs@@3P6AHPEAU_RTL_CONDITION_VARIABLE@@PEAU_RTL_CRITICAL_SECTION@@K@ZEA 0000000180026248     MSVCRT:thread_safe_statics.obj
 0003:0001b250       ?g_wake_all_condition_variable@@3P6AXPEAU_RTL_CONDITION_VARIABLE@@@ZEA 0000000180026250     MSVCRT:thread_safe_statics.obj
 0003:0001b25c       ?__proc_attached@@3HA      000000018002625c     MSVCRT:dll_dllmain.obj
 0003:0001b270       ?is_initialized_as_dll@@3_NA 0000000180026270     MSVCRT:utility.obj
 0003:0001b271       ?module_local_atexit_table_initialized@@3_NA 0000000180026271     MSVCRT:utility.obj
 0003:0001b278       ?module_local_atexit_table@@3U_onexit_table_t@@A 0000000180026278     MSVCRT:utility.obj
 0003:0001b290       ?module_local_at_quick_exit_table@@3U_onexit_table_t@@A 0000000180026290     MSVCRT:utility.obj
